:106E070047415445202D3E49533A200047415445B8
:086E1700202D3E52463A2000F6
:106EBE007B017A007980227B017A007900900100B3
:036ECE00E0FD22C2
:10650B0030003BC200D211C2A1E4FF1209FBEF64C1
:10651B00017029126EBE122AB8C296126EBE1240BC
:10652B00AA126EBE126FE07BFF7A6E7907E4FD1242
:0F653B003AF9126EBEE4FD123AF9D296D2A122BD
:10668100300137C201C211C2A1E4FF1209FBEF645C
:10669100017025126EC5125C03126EC51243A7125A
:1066A1006EBE122AB87BFF7A6E7913E4FD123AF9B5
:0B66B100126EBEE4FD123AF9D2A122E5
:1066F6000D0A494F31202D3E544E433A200057583B
:1067060020426F617264206E6F206C696E6B0D0A99
:106716000041504757314B0041504757314B0054C9
:076726004350495020000020
:10530800EF9325E0FF90020FE02400F582E43400DB
:10531800F583EFF090020FE004F022E025E044600E
:10532800FF90020FE02400F582E43400F58322EFB9
:10533800F090020EE004F02290020EE0FFC3940603
:1053480022EFF0900211E004F022A3F0E490020EA4
:10535800F022900210E004F02290020EE02418F5EA
:1053680082E43402F5832290020EE02421F582E4DF
:105378003402F5832290020EE0244AF582E43403D5
:10538800F583E0FF2274032FF582E43401F583E00E
:0153980022F2
:106DEE00308315E4FFFE126E64EF600C12650B1219
:096DFE0066811263FA126440225E
:0509FB0090020DEFF079
:100A0000E490020FF0EF701490020EF01253405079
:100A10002090671E12530812533980F0E490020EA2
:100A2000F0125340500B906717125308125339803D
:100A3000F0125329746012531BE490020EF012530B
:100A40004050277E00126E64900217EFF07008127B
:100A500053297440F0800B900217E025E0125328D0
:100A6000EFF012531C12533980D490020DE0700540
:100A70007F87FE80047F077E01126E64900216EF6E
:100A8000F0201103301229900216E025E044E01214
:100A9000530CE490020EF0125340500CEF90672577
:100AA00012530912533980EF12532974E1020BAB30
:100AB00090020DE0900212701204F0A37490F07F87
:100AC00096120E227497F07F9D80117401F0A3742A
:100AD000A0F07FA6120E2274A7F07FAD7E01126EE9
:100AE00064900229EFF0900216E025E044E01253F2
:100AF00028EFF0900212120E34605112531CE49051
:100B0000020EF01253405023900213E09002121292
:100B10000E1370081253617420F0800A900217E0DF
:100B2000FF125361EFF012533980D8E490020EF0B7
:100B3000125340500F74182F125367E012530A12C9
:100B4000533980EC900220125323EFF090021412DC
:100B50000E34605112531CE490020EF012534050B8
:100B600023900215E0900214120E13700812536FB6
:100B70007420F0800A900217E0FF12536FEFF0121A
:100B8000533980D8E490020EF0125340500F742174
:100B90002F125375E012530A12533980EC90022938
:100BA000125323EFF0125329E0440112531B125346
:100BB00029740312531B12532C74F012531B90020E
:100BC0000DE06003020C7A7F88FE126E6412530DF2
:100BD000A3E4F07490125352120DBB1253497003E8
:100BE00012535A12531C125339E0C3940840E97F40
:100BF000897E00126E6412530DA3E4F074A01253A8
:100C000052120DBB125349700312535A12531C1245
:100C10005339E0C3940940E97F8A7E00126E641262
:100C2000530DA3E4F0A374B0125353120E066017D1
:100C3000120DD4125349700312535A12531C1253FB
:100C400039E0D3941F40E47F857E00126E64EF6428
:100C5000016003020DAD125329742012531B12516F
:100C6000E0E490020EF012537D600C1253291253EF
:100C700037A3E004F080EF020DAD90020DE06401B7
:100C80006003020DB87F087E01126E6412530DA33B
:100C90007401F0A37410125353120DD412534970FF
:100CA0000312535A12531C125339E0C3940840E9FB
:100CB0007F097E01126E6412530DA37401F0A374B8
:100CC00020125353120DED125349700312535A124E
:100CD000531C125339E0C3940940E97F0A7E011284
:100CE0006E6412530DE4FF125C6FEF701D7BFF7A90
:100CF0006679F6FD123AF97A677904120E3E7A00A7
:100D00007980E4FD1215977F00227A6679F6120E3B
:100D10003E7A017903E4FD123AF990020E7401F073
:100D200090020EE0FFC39404500B12538D12530C2B
:100D300012533980EB125329742F12531B90020E59
:100D40007405F090020EE0FFC39421500B12538DF6
:100D500012530C12533980EB9002107401F0A374FB
:100D600030125353120E066017120DED12534970D4
:100D70000312535A12531C125339E0D3941F40E408
:100D80007F057E01126E64EF640170211253297495
:100D90002012531B1251E0E490020EF012537D60BA
:100DA0000C125329125337A3E004F080EF90020F86
:0A0DB000E0900100F07F01227F00B7
:100DBA0022900210E0FEA3E0FF126E6490020FE0A0
:100DCA002400F582E43400F58322900210E0FEA3A9
:100DDA00E0FF126E6490020FE02400F582E4340012
:100DEA00F58322900210E0FEA3E0FF126E649002E7
:100DFA000FE02400F582E43400F58322900210E02B
:100E0A00FEA3E0FF126E64EF222FFFE03400FE1211
:100E1A006E64900217EFF0227E01126E6490022037
:100E2A00EFF09002147401F0A322E0FEA3E0FF1297
:0E0E3A006E64EF227BFFE4FD123AF97B012289
:100026000D0A575820202D3E4953203A20000D0A2C
:0C003600575820202D3E5246203A200052
:106ED1007B017A007980227B017A007900900100A0
:036EE100E0FD22AF
:1063FA00300442C204D212C2A17F011209FBEF6427
:10640A00017030126ED1122AB8126ED11240AA123D
:10641A006ED1126FE07BFF7A007926E4FD123AF919
:10642A00126ED1E4FD123AF97B017A0179037D01FA
:06643A00121597D2A12209
:106B5100900103E064636007E4900185F0FF2290F7
:106B61000185E064246004E4F0FF2290037874015D
:076B7100F0E4F5AF7F012203
:10644000300342C203C212C2A17F011209FBEF64F2
:10645000017030126ED8125C03126ED81243A7126C
:106460006ED1122AB87BFF7A007934E4FD123AF932
:10647000126ED1E4FD123AF97B017A0179037D01B4
:06648000121597D2A122C3
:055C6F0090023DEFF082
:105C7400E4F5AF90018404F0759CF4E4F5A290037C
:105C840078F0900185F090023EF090023EE0FFC370
:105C94009480501474032FF582E43401F583E4F006
:105CA40090023EE004F080E275AF01E490023EF021
:105CB400900378E070177F02FE126D1290023EE0AE
:105CC40004F0E0D3946440E8E4F5AFFF22E4F5AFD8
:025CD4007F014E
:015CD60022AB
:106CB800202020202020202020202020200D0A0015
:0E6CC8004750532D3E42454143454E3A200071
:106B9F00900100E0FF90037DE0FEC39F2274002E62
:106BAF00F582E43400F583E0FF227B017A0079005F
:066BBF00900100E0FD2240
:10486200C2A112493B7F031209FB126BB9125C030E
:10487200126BB91243A77FC0120003E4FF120003B8
:10488200E490037DF0126B9F500E126BAC1200038A
:1048920090037DE004F080ED7FC01200037B017A7B
:1048A200007980122AB87B017A0079801240AA7BB3
:1048B200FF7A6C79C8124925124925126FE07F846C
:1048C2007E01126E64EF14600E146026146046249A
:1048D200037047E4FF8040E490037DF090037DE0A5
:1048E2002480F582E43400F583E0FF602D12493123
:1048F20080EA7FC0126E4DE4FF126E4DE490037D9C
:10490200F0126B9F5008126BAC12493180F37FC0DA
:10491200126E4D80057F01123F9012493B122C808E
:02492200D2A120
:1049240022E4FD123AF97B017A00798022126E4D5D
:1049340090037DE004F0227BFF7A6C79B8E4FD12E9
:034944003AF9221B
:104D31000D0A50494E47204641494C2C5345525685
:104D41004552204F46464C494E45200D0A000D0A5A
:104D5100534552564552204C494E4B2053544152D3
:104D6100542E2E2E0D0A0053455256455220434CC7
:104D71004F534520210D0A005345525645522054A8
:104D810043502F4950204C494E4B204F55545449C4
:104D91004D45210D0A00534552564552205443506A
:104DA1002F4950204C494E4B204F555454494D45A5
:104DB100203E2033202C4E6F7720544E43205265E5
:104DC10073657420210D0A007573657220002070CF
:104DD100617373200020566572732047573130305C
:074DE10030203130382000C2
:1056540090022BE02480F582E43400F5832290024A
:105664001CE0FEA3E0FF90021AE0FCA3E0FD900220
:1056740017E02DFD900216E03CFC22F090022BE096
:1056840004F022EFF090022AE004F0A3E004F022F8
:105694009002107404F0A3E4F0223400FEF0A3EFAF
:1056A400F0EE5407FEE42FFFEE344022FF90021C7C
:1056B400E03400FE22EFF0900227E004F0223400F0
:1056C400F0A3CEF022900226E004F022900226E419
:0356D400F0A3221E
:102FE40090021C1256972402FFE43404FE1268F384
:102FF400900212EFF07D0212000EEF6401600302F2
:10300400315990021DE024021256B0900212E0449D
:1030140004FD126BCC90021DE0242612315A7F006D
:10302400FEC006C00790021DE0242712315AFDD0CD
:10303400E02DFED0E090021A1256C290021DE02448
:10304400281256B01268F3EF7F00FEC006C0079046
:10305400021DE024291256B01268F3EFFDD0E02DD2
:10306400FED0E09002161256C2D390021BE0948068
:1030740090021AE0940040061256620265C890025B
:1030840016E05407FEA3E02400FFEE3460A3F0A38F
:10309400EFF0A3E0FFA3E0900214CFF0A3EFF0E47D
:1030A400900213F0900214E07002A3E0604C9002CE
:1030B40018E0FEA3E0FF1268F3900213125657EFD4
:1030C400F0900219E004F07006900218E004F09009
:1030D4000213E004F0900215E024FFF0900214E0E3
:1030E40034FFF0900218E0B468BAA3E0B400B590DD
:1030F40002187460F0A3E4F080AA900213125657E9
:10310400E4F01256621265C87B017A007980E4FD0E
:10311400123AF9900080E06423703390035AF0204F
:103124000A33900213F0FF900213125657E0FE6028
:103134000EB420010F900213E004F0EFB403E89002
:103144000213125657E0B47602D20A021E1AC2A122
:053154001239C6D2A1F2
:0E31590022FF90021CE03400FE1268F3EF2209
:106F1C0090035AE004F0E0D3943C4004E4F0D20B2C
:016F2C002242
:106CD600900359E0FFB4020F0512E512D394024067
:0E6CE6000CE4F512B2B722EFB40302B2B722EB
:106CF400123C2490035B7413F0A37488F0751301A1
:0E6D0400E4900358F0A3F0F512A3F0C20B22A6
:106A0000E4FFFE126E6490020DEFF07F097E00122B
:106A10006E6420810C90020DE06006EF6003022698
:0A6A2000C8E4900359F0D2B7D296F3
:016A2A002249
:1068640090035CE004F0700690035BE004F0D390C6
:10687400035CE0948D90035BE0941340137413F075
:10688400A37488F00513E513D3940340037513012F
:0168940022E1
:1026C800125694300B1590035AF0C20B126864E44A
:1026D800900359F07A4D79311228C0900359E0607F
:1026E800030227E27A4D794F1228C0125694D2B7C6
:1026F800C209C20A90035AF0C20BFF12289890032D
:102708005BE0FD7404FFFE126BCC90035BA3E0FD5D
:102718007F057E04126BCC7F0112289812288B64E7
:102728001360030227D97F2FFE126E64EF640170D5
:10273800057F22FE800DE51324FE602304703C7F94
:10274800227E00126E64AD071228A07F231228573C
:102758001228A87F241228571228B07F2580427F8C
:102768002612287B1228A07F2712287B1228A87FF0
:10277800281228831228B07F2980267F2A122883CE
:102788007F0C7E04126BCC7F2B1228B87F0D7E0441
:10279800126BCC7F2C1228B87F0E7E04126BCC7F74
:1027A8002D7E00126E64AD077F0F7E04126BCC7D08
:1027B800387F107E04126BCC7DF47F117E04126B7F
:1027C800CC7D047F017E04126BCC9003597401F018
:1027D800227D107F017E04026BCC12288BBF171359
:1027E800900359200A057403F080057405F0C2B7F8
:1027F800022FE49003597402F0FF7E041268F390EC
:10280800020FEFF030E10EE0440212285F7A4D79B2
:1028180068FD023AF990020FE030E33244081228CA
:102828005F7A4D7979FD123AF97F307E00126E6435
:10283800BF011B900358E004F0E0D39403400FE479
:0E284800F07BFF7A4D7997FD123AF975C720A3
:10285600227E00126E64AD0722FD7F027E04126B9B
:10286600CC7D107F017E04126BCC126864E4900369
:1028760059F07BFF227E00126E64AD07227E0012A5
:102886006E64AD07227F037E041268F390020EEF9A
:10289600F0227D017E04126BCC227F0C7E04126B2B
:1028A600CC227F0D7E04126BCC227F0E7E04126B2F
:1028B600CC227E00126E64AD07227BFFFD123AF930
:0128C60022EF
:101E1A00300903022028E4FFFE126E64EF70030209
:101E2A0020287F0912205A7003022028E490022BEE
:101E3A00F090022AF090022AE0904DC993FF6008C0
:101E4A0012565412568780EDE4900226F0A3F0123F
:101E5A002029EF60131220291256541256B9700322
:101E6A001256C912568080E77F0712205A60301234
:101E7A005654742D12567FEFC3940AEF5002801500
:101E8A0075F00A842430FE125654EE12567FEF750E
:101E9A00F00A84E5F02430FF125657EF12567FE419
:101EAA0090022AF090022AE0904DCF93FF60081228
:101EBA00565412568780ED1256D07409F012203506
:101ECA00EF60131220351256541256B97003125687
:101EDA00C912568080E7E490022AF090022AE09024
:101EEA004DD693FF600812565412568780ED12564B
:101EFA00D07440F0FF7E00126E64EFC394FF501F4F
:101F0A001256D07440F012204EEF601312204E1277
:101F1A0056541256B970031256C912568080E712E7
:101F2A005654740D12567F125657740A12567F125F
:101F3A005657E4F09002281256972420FFE43404FE
:101F4A00FE1268F3EF7F00FEC006C007900229E088
:101F5A002421122041FDD0E02DFED0E03400900271
:101F6A0020F0A3CEF0900229E024241220417F0021
:101F7A00FEC006C007900229E02425FF900228E04F
:101F8A003400FE1268F3EFFDD0E02DFFD0E090029E
:101F9A001E12569E900222F0A3EFF0E4A3F0A3F0E3
:101FAA0090022AF090022A125657E0FD60449002ED
:101FBA0022E0FEA3E0FF126BCC900223E004F07053
:101FCA0006900222E004F090022AE004F090022532
:101FDA00E004F07006900224E004F0900222E0B4DB
:101FEA0048C2A3E0B400BD9002227440F0A3E4F01A
:101FFA0080B2900228E0FEA3E0FF900224E0FCA356
:10200A00E0FD90021FE02DFD90021EE03CFC1267ED
:0E201A00647B017A007980E4FD123AF9D20964
:1020280022900226E0FEA3E0FF126E6422900226B0
:10203800E0FEA3E0FF126E6422FF900228E0340065
:10204800FE1268F3EF22900226E0FEA3E0FF126E74
:0920580064227E00126E64EF2286
:0B40AA0090020FEBF0A3EAF0A3E9F096
:1040B500900359E0640560030241AAC29690021A72
:1040C5001256972420FFE43404FE1268F3EF7F00B4
:1040D500FEC006C00790021BE024211241ABFDD0B3
:1040E500E02DFED0E03400900216F0A3CEF0900251
:1040F5001BE024241241AB7F00FEC006C0079002DE
:104105001BE02425FF90021AE03400FE1268F3EF4D
:10411500FDD0E02DFFD0E090021412569E900218BB
:10412500F0A3EFF0E4900212F0A3F090020FE0FB91
:10413500A3E0FAA3E0F9120301FD6048900218E03C
:10414500FEA3E0FF126BCC900219E004F07006901C
:104155000218E004F0900210E475F0011203D0900B
:104165000213E004F07006900212E004F0900218C9
:10417500E0B448B7A3E0B400B29002187440F0A3CD
:10418500E4F080A790021AE0FEA3E0FF900212E09F
:10419500FCA3E0FD900215E02DFD900214E03CFC2F
:0541A500126764D296D0
:0E41AA0022FF90021AE03400FE1268F3EF22AA
:105759002352455345540023494E5354414C4C0060
:1057690023474154455F52465F54455354002347EC
:105779004154455F49535F54455354002357585F7B
:1057890052465F54455354002357585F49535F5459
:10579900455354002348454C4C4F000D0A00632ED5
:1057A9002E2E732E2E2E672E2E2E742E2E2E722E08
:1057B9002E2E702E2E2E682E2E622E2E2E2E2E0D71
:1057C9000A002348454C4C4F00000000000000002F
:0157D90000CF
:1056D700900212E05407FEA3E02400FFEE3470901E
:1056E700036CF0A3EFF02290022DE0FBA3E0FAA3F6
:1056F700E0F902030190022DE475F0010203D034B2
:1057070000FEF0A3EFF0EE5407FEE42FFFEE345057
:1057170022FF90022BE03400FE2290036CF0A3E4FA
:10572700F022EBF0A3EAF0A3E9F0227406F0A3E479
:10573700F02420FFE43406FE22E490036BF0C2134A
:10574700223400F0A3CEF0229002357450F0A3E487
:02575700F0223E
:0A7004002081030253991257402225
:03704A00C213224C
:101B8300781C7C027D017BFF7A5779CB7E007F0F27
:101B93001202DB90022B7406F0A3E4F02402FFE4AC
:101BA3003406FE1268F3900210EFF07D0212000E6D
:101BB300EF64016003021DC190022CE0240212575E
:101BC30018900210E04404FD126BCC90022CE02428
:101BD30026121DFE7F00FEC006C00790022CE024E3
:101BE30027121DFEFDD0E02DFED0E0900214125707
:101BF3004890022CE024281257181268F3EF7F0054
:101C0300FEC006C00790022CE02429125718126860
:101C1300F3EFFDD0E02DFFD0E03400FE900212F090
:101C2300A3EFF0900215E02FFF900214E03E900224
:101C330016F0A3EFF07FF07E01126E64900222EFA4
:101C4300F07FF17E01126E64900223EFF07FF27E4B
:101C530001126E64900224EFF07FF37E01126E6432
:101C6300900225EFF07FF47E01126E64900226EF5E
:101C7300F07FF57E01126E64900227EFF07FF67E0F
:101C830001126E64900228EFF07FF77E01126E64FA
:101C9300900229EFF0E4A3F01256D77B017A027980
:101CA3001C126C30EF6401707C900214E07004A38A
:101CB300E0640E700BC2AC121DC212229AD2AC2287
:101CC300900214E064027004A3E0640E7057C2AF84
:101CD300C2A0C2A1FFFE126EE4E490021AF0A3F0C8
:101CE300900218F0A3F0126A2B900211EFF0FD900E
:101CF300021AE0FEA3E0FF12684890021BE004F022
:101D0300700690021AE004F0900219E004F07006E5
:101D1300900218E004F0C3900218E0940240C71246
:101D23001DC275C7201256D77BFF7A577959126C9B
:101D330030BF0106121DD675C7201256D77BFF7A16
:101D4300577960126C30BF0109121DD612206175DC
:101D5300C7201256D77BFF7A577969126C30BF01BF
:101D630006121DEAD201221256D77BFF7A577977E2
:101D7300126C30BF0106121DEAD200221256D77B25
:101D8300FF7A577985126C30BF010B90022BE0FE6E
:101D9300121E0BD203221256D77BFF7A5779911268
:101DA3006C3090022BE0FEBF0106121E0BD2042200
:0E1DB300A3E0FF900216E0FCA3E0FD1265C85D
:101DC1002290022BE0FEA3E0FF900216E0FCA3E0CC
:101DD100FD1265C82290022BE0FEA3E0FF900216DF
:101DE100E0FCA3E0FD1265C82290022BE0FEA3E017
:101DF100FF900216E0FCA3E0FD1265C822FF9002ED
:101E01002BE03400FE1268F3EF22A3E0FF900216EC
:091E1100E0FCA3E0FD1265C8220B
:106A2B0090036CE0FEA3E0FF1268F390036DE004AB
:106A3B00F0700690036CE004F090036CE0B4780AFD
:0A6A4B00A3E0B40005747012572197
:016A5500221E
:10692100AD0790036CE0FEA3E0FF126BCC90036D0A
:10693100E004F0700690036CE004F090036CE0B4A6
:0D694100580AA3E0B400057450125721223B
:106C300090022D1257291256EE6014126A2B12562A
:106C4000EE6F60037F002290022E1256FF80E77FD6
:026C500001221F
:066AD60090023D12572959
:106ADC00E4A3F090023D1256F1FF6011126921906F
:106AEC00023E1256FF900240E004F080E690024015
:026AFC00E0FFB9
:016AFE002275
:10229A00C29690023B1257321268F3EF7F00FEC0DB
:1022AA0006C00790023CE02421122490FDD0E02DC4
:1022BA00FED0E090023912574890023CE0242412E2
:1022CA0024907F00FEC006C00790023CE02425FF50
:1022DA0090023BE03400FE1268F3EFFDD0E02DFFE0
:1022EA00D0E09002371257061256E6E4900231F017
:1022FA00A3F07BFF7A57799D12249DE4900233F074
:10230A00A3F090022FF0A3F0900233E0FEA3E0FFC7
:10231A00126E6490022DEFF0126921900234E004EB
:10232A00F07006900233E004F0900230E004F0709E
:10233A000690022FE004F0C390022FE0940240C8F6
:10234A00900232E02400F0900231E03402F07A6A1E
:10235A0079671224B3EFF07A5779A41224B3E00410
:10236A00F0E004F0E51312241DE490022EF090032D
:10237A005BE0FEA3E0FF900235EEF0A3EFF07C03F2
:10238A007DE812037BEF1224BCF07D6412244B7D9E
:10239A000A12244B900235E0FEA3E0FF7C007D0A7E
:1023AA0012037BED12241DE490022EF0900359E0F3
:1023BA001224BC12246D1264CAEF64017017FF1252
:1023CA005C6FBF01087B017A017903800E7BFF7A7B
:1023DA005779A780067BFF7A5779A712249D125155
:1023EA00E07B017A03794A126AD690022EEF122410
:1023FA006D90023BE0FEA3E0FF900231E0FCA3E017
:10240A00FD900238E02DFD900237E03CFC12676433
:02241A00D29658
:10241C00222430FF12692190022EE004F07BFF7A17
:10242C005779A4126AD690022EE004F0E004F0E092
:10243C00FF900232E02FF0900231E03400F0229055
:10244C000235E0FEA3E0FF7C0012037B7C007D0ADA
:10245C0012037BED2430FF12692190022EE004F070
:10246C0022F07BFF7A5779A4126AD690022EE004F0
:10247C00F0E004F0E0FF900232E02FF0900231E047
:10248C003400F022FF90023BE03400FE1268F3EFC0
:10249C0022126AD690022EEFF0900232E02FF090CA
:1024AC000231E03400F0227BFF126AD690022E2219
:0C24BC002430FF12692190022EE004225F
:1064CA007F0012650140037F01227401FFFE126EF4
:1064DA0064EFD3940040037F01227F0212650140DA
:1064EA00037F01227F037E01126E64EFD394004082
:1064FA00037F01227F00227E01126E64EFD3940093
:01650A00226E
:1053990090020E7406F0A3E4F020133C125741D298
:1053A900967D01FF7E06126BCC7DEA7F047E061294
:1053B9006BCC7D607F057E06126BCC7D0112541586
:1053C900BF130C7D021254156414703FD213227D51
:1053D900107F017E06026BCC7F037E061268F39074
:1053E900020DEFF0601724E4600F2405701D90038F
:1053F9006B7401F0C296021B837D0880027D107FC9
:0B540900017E06126BCC125740D296B9
:10541400227F017E06126BCC7F037E061268F39016
:05542400020DEFF02273
:093AF90090022C125729A3EDF0F4
:103B020090036BE07003023C0C90023712573212A2
:103B120068F3EF7F00FEC006C007900238E0242160
:103B2200123C0DFDD0E02DFED0E03400900233F0C7
:103B3200A3CEF0900238E02424123C0D7F00FEC098
:103B420006C007900238E02425FF900237E03400D7
:103B5200FE1268F3EFFDD0E02DFFD0E090023112AB
:103B62005706900235F0A3EFF090022FE07038A3D1
:103B7200F090022C1256F1FD6073900235E0FEA324
:103B8200E0FF123C1A7006900235E004F01256FC77
:103B9200900230E004F0900235E0B458D4A3E0B4CF
:103BA20000CF12574F80CA90022FE0A3F09002304C
:103BB200E06034900235E0FEA3E0FF90022C125642
:103BC200F1FD123C1A7006900235E004F01256FC28
:103BD200900230E014F0900235E0B458D0A3E0B483
:103BE20000CB12574F80C690022FE0A3F09002370D
:103BF200E0FEA3E0FF900230E0FD900232E02DFDF6
:0A3C0200900231E03400FC12676408
:103C0C0022FF900237E03400FE1268F3EF22126BB1
:083C1C00CC900236E004F02216
:09700E00FF900360E03400FE2253
:0C6FD4002081030257DAE490037EF022D3
:06704000E490037EF02243
:104AE7009003607407F0A3E4F02402FFE43407FEA8
:104AF7001268F390035DEFF07D0212000EEF640180
:104B07006003024B9E900361E0240212700E900333
:104B17005DE04404FD126BCC900361E02426124B48
:104B27009F7F00FEC006C007900361E02427124B59
:104B37009FFDD0E02DFED0E0340090035EF0A3CEC1
:104B4700F0900361E0242812700E1268F3EF7F00E3
:104B5700FEC006C007900361E0242912700E126898
:104B6700F3EFFDD0E02DFFD0E03400AD07FC540794
:104B7700FEE42FFFEE3478FEE4B50704EEB48000C0
:104B8700900360E0FEA3E0FF90035FE02DFD90033C
:074B97005EE03CFC1265C862
:0E4B9E0022FF900360E03400FE1268F3EF2265
:1057DA007F317E00126E64EF60769003697407F081
:1057EA00A3E4F090037EE0703F7D02FF7E07126B18
:1057FA00CC7DEA7F047E07126BCC7D6A7F057E072B
:10580A00126BCC7D017F017E07126BCC7F037E0772
:10581A001268F3BF220990037E7401F0024AE77D01
:10582A00107F017E07026BCC7F027E071268F3EFBE
:10583A0030E31D900367A3E04408FD7F027E071250
:10584A006BCC7D107F017E07126BCCE490037EF057
:01585A00222B
:0B6FE00090020DEBF0A3EAF0A3E9F033
:016FEB002283
:09701700FF90023DE03400FE226E
:10000E00AE05EFA806088002C313D8FC30E0037FCC
:05001E0001227F002219
:103C2400D294C290C280126F5AD2807F10123D0F7C
:103C34007F0F7E00126BCC7F11123D0F7F107E0030
:103C4400126BCC7F12123D177F117E00126BCC7F5A
:103C540013123D177F127E00126BCC7F14123D1F8E
:103C64007F057E00126BCC7F15123D1F7F067E0000
:103C7400126BCC7F16123D277F077E00126BCC7F20
:103C840017123D277F087E00126BCC7F18123D2F40
:103C94007F017E00126BCC7F19123D2F7F027E00C4
:103CA400126BCC7F1A123D377F037E00126BCC7FE0
:103CB4001B123D377F047E00126BCC7F1C123D3FEC
:103CC4007F097E00126BCC7F1D123D3F7F0A7E0070
:103CD400126BCC7F1E123D477F0B7E00126BCC7F94
:103CE4001F123D477F0C7E00126BCC7F207E00129A
:103CF4006E64AD077F0D7E00126BCC7F217E0012B7
:103D04006E64AD077F0E7E00026BCC7E00126E6483
:103D1400AD07227E00126E64AD07227E00126E642F
:103D2400AD07227E00126E64AD07227E00126E641F
:103D3400AD07227E00126E64AD07227E00126E640F
:0B3D4400AD07227E00126E64AD072266
:0E6F5A00E4F5D875F9FDF5E9D2DE30DFFD2251
:106DBA00E4FEEF30E704D2918002C291D290EF252F
:096DCA00E0FFC2900EEEB408E9EE
:016DD300229D
:076BC500FFE43EFEA3E0FD2A
:106BCC00AB07AA06C2947FF0126DBAEAFF126DBA37
:0D6BDC00AF03126DBAAF05126DBAD294224C
:0468F300AD07AC063B
:1068F700C2947F0F126DBAECFF126DBAAF05126D1D
:10690700BAE4FFFED290EF25E0FF3093034401FF86
:09691700C2900EEEB408EDD2941A
:016920002254
:1067640090023FECF0A3EDF090023DEEF0A3EFF0C9
:106774002424126BC590023EE02425127017900267
:1067840040E0FD126BCC90023EE024011270177DB4
:0467940020026BCCA8
:1065C80090022FECF0A3EDF090022DEEF0A3EFF087
:1065D8002428126BC590022EE02429FF90022DE09A
:1065E8003400FE900230E0FD126BCC90022EE024C5
:0E65F80001FF90022DE03400FE7D40026BCCCE
:10623A00E0FAA3E0FBFFAE0212037BEF2430FF90EB
:10624A00020DE0242CF582E43403F583EFF090028A
:10625A000DE004F0227C00AF03AE0212037B7C0047
:10626A007D0A12037BED22E0242CF582E43403F547
:0D627A008322E0FAA3E0FB7C007D0AFF22F6
:10345A00126AACEF7002FF227FCC126D307F4412E9
:10346A006D3030C6FD126AACEF7002FF227FCC12BB
:10347A006D307FBE126D30126C52900334E4F0A3AB
:10348A00EFF0126C52900332E4F0A3EFF0E49002F2
:10349A000DF090020DE0FFC39406500C742C2F120D
:1034AA006274E412625780EA900332A3E0FF30E7C5
:1034BA001DD214FE900335E02400FF900334E03E51
:1034CA00FEEFF4FFEEF4FEEF2401FDE48012C214D5
:1034DA00900333E0FE900335E02400FD900334E0CE
:1034EA003EFCE4120151E4FBFA7920783F120046CF
:1034FA0012018A90020EEEF0A3EFF0E490020DF0B2
:10350A00301408126271742D126257C390020FE0D0
:10351A00946490020EE09400500C12627CAE021287
:10352A00037BEF023593C390020FE094E890020EFA
:10353A00E09403502C7C007D6412623A7D0A126288
:10354A005F2430FF12624C126271742E126257A30A
:10355A00E0FEA3E0FF1262682430FF90020D0235FC
:10356A00ADC390020FE0941090020EE094275041F0
:10357A007C037DE812623A7D6412625F2430FF1296
:10358A00624CA312627C1262631262461262717406
:10359A002E1262577C007D0AAF03AE0212037BED46
:1035AA002430FF12624C12627174431262577F0117
:0335BA00227F006D
:0135BD0022EB
:076F0A00126F11D2C67F01D6
:0B6F1100AE071FEE6004000080F622B7
:106AAC00D2D7C2C67FF0126F117FF0126F11D2C60F
:106ABC007F3C126F11A2C67FF0126F117FB4126F60
:0A6ACC001120D7037F01227F002272
:106C5200E4FDFCEDC313FDC2C67F01126F0A30C60C
:106C620004ED4480FD7F3C126F110CECB408E4AFDC
:016C7200051C
:016C730022FE
:026D3000AD07AD
:106D3200E4FCC2C67F01126F11EDC313FD92C67F40
:096D42003C126F0A0CECB408E9E4
:016D4B002225
:0D6FAD000D0A495320202D3E52463A200087
:10660600F00C74002CF582E43400F58374A0F00CD1
:1066160074002CF582E43400F5832274802DF58213
:10662600E43400F583E02274812EF582E43400F52B
:0E66360083E022EEF00C90021EE004F00D2234
:10609D00E4FF74802F126624643E600A0FEFD394E0
:1060AD000C40EF7F6322E4FE74802E126624FD64A3
:1060BD003E6030ED642D7028C3EF9EB40208126669
:1060CD002DC39430FF2212662D24D075F00AA4FF43
:1060DD0074822EF582E43400F583E024D02FFF2264
:0560ED000E80C57F00DC
:0160F200228B
:0D6FA0007F2E7E00126E6490037FEFF022C2
:1039C60090037FE07003023AF812609DEF64637023
:1039D60003023AF8E4FE74802E126624643E600800
:1039E6000EEED3940C40EF227D069000007440F05A
:1039F600A3DDFC7D060EE4FC74802E126624FB64B7
:103A06002C6012EB25E0FB126616EBF00C0EEED3E3
:103A1600941240E4229000067460F00C7D0690003B
:103A2600077440F0A3DDFC7C07EFD39400401AE452
:103A3600FD90021EF0126621FE642D6026EE25E042
:103A4600FE12661612663980ECE4FD90021EF01234
:103A56006621FE643E600CEE25E0FE1266161266D6
:103A66003980ECEF25E0446090000DF07C0E126684
:103A76001674A81266147486126606749212660686
:103A8600744012661474E112661474031266147498
:103A9600F0F00CE4FD126621643A60080DEDD39453
:103AA6003240F2220D126621FF6009126616EFF00F
:103AB6000C0D80F1AF04900100EFF0FD7B017A0060
:103AC6007900125C037B017A007900900100E0FD29
:103AD6001243A77B017A007980122AB87BFF7A6F9E
:103AE60079ADE4FD123AF97B017A007980E4FD12A2
:023AF6003AF99B
:013AF80022AB
:105AB900E0FF90021FE0FBA3E0FAA3E0F9900223C4
:105AC900E0F58275830022EF120347900223E00478
:105AD900F022EF4430FFF090021FE0FBA3E0FAA3AD
:105AE900E0F92274002FF582E43400F583E0C31352
:105AF900900225F0642022E0541EC313900226F080
:105B0900D3940022900226E024F6F0E044302224C7
:105B190006F582E43400F58322900222E004F022A3
:0B2AB80090021FEBF0A3EAF0A3E9F08E
:102AC300E4900223F09002227407F0900222E0FFC8
:102AD300C3940D5010125AEC6006125AB9125AD010
:102AE300125B2280E690000D125B00402A125ABB53
:102AF300742D125AD1900226E0FFC3940A50051296
:102B03005ADB800D125ABB7431125AD1125B0DFF7E
:102B1300F0125AC6125AD0125ABB743E125AD1E45A
:102B2300900222F0900222E0FFC394065010125A42
:102B3300EC6006125AB9125AD0125B2280E690005A
:102B430006125B00402A125ABB742D125AD190020E
:102B530026E0FFC3940A5005125ADB800D125ABBBC
:102B63007431125AD1125B0DFFF0125AC6125AD0A9
:102B73009002247407F090000DE030E003022C1E55
:102B8300125ABB742C125AD1A3E02407F0E090022E
:102B930022F0900224E02406FFE433FE900222E0B8
:102BA300FDC39FEE6480F8748098501374002D1257
:102BB3005AEF6006125AB9125AD0125B2280D39090
:102BC3000224E0FF125B18125B00402F125ABB7401
:102BD3002D125AD1900226E0FEC3940A5009EE4406
:102BE30030FE125ADF800D125ABB7431125AD112C1
:102BF3005B0DFEF0125AC6EE125AD174062F125B09
:102C03001AE030E708125ABB742A125AD1900224F0
:102C1300E0125B18E020E003022B83125ABB743AE4
:102C2300125AD1A3E02409F0E0900222F0900100AF
:102C3300E0FF900222E0FEC39F502B74002EF5822A
:102C4300E43400F583125AB9125AD0E0FFD39478D2
:102C5300400F125AE08F82758300747E125AD1801E
:102C630005125B2280C7125ABB740D125AD1125A35
:0D2C7300C9740A125AD1125AC9E40203476B
:106D4C000D0A4E4D45412039363030204F55543ABE
:0C6D5C00200024475057504C2C00000031
:106C74000FE0FE74802FF582E43400F583EEF00F0C
:106C840074802FF582E43400F583227B017A007945
:026C940080225C
:053F900090020FEFF0AC
:103F950078107C027D017BFF7A6D795E7E007F0A59
:103FA5001202DBE4FFFE74102EF582E43402F58381
:103FB500E0FD126C84EDF00F0EEEB407E9E4FE743B
:103FC5007F2EF582E43402F583E0FD126C84EDF07A
:103FD5000F0EEEB407E9126C84742CF09002B9123E
:103FE5006C74742CF00FE4FE74742EF582E43402C4
:103FF500F583E0FD126C84EDF00F0EEEB408E912C6
:104005006C84742CF09002B8126C74742CF00FE46C
:10401500FE748A2EF582E43402F583E0FD60091210
:104025006C84EDF00F0E80E9126C84742AF00FE4B5
:10403500FD7E01EF14FCEEC39C500C74802E126CB7
:1040450087E06DFD0E80ECEDC4540FFEC3940AEEBF
:104055005004243080022437FE126C84EEF00FEDFC
:10406500540FFEC3940AEE5004243080022437FE18
:10407500126C84EEF00F126C84740D126C82740A4B
:10408500126C82E4F0126C8F1267FF126C8F12674C
:10409500CC7BFF7A6D794CE4FD123AF9126C8FE412
:0440A500FD123AF9D5
:0140A90022F4
:106E1F000D0A524620494E203A20000D0A495320B0
:076E2F004F5554203A2000EA
:106DD400900100E0FF90020EE0FEC39F2274002E9B
:0A6DE400F582E43400F583E0FF229D
:104F5300C2A07B017A007980122AB87A6E791F1277
:104F63004FF6E4FD123AF97F357E00126E64BF01FD
:104F7300157B017A0079801240AA7A6E792A124F42
:104F8300F6E4FD123AF9126D687F847E01126E64B5
:104F9300BF01077F02123F90804E7FC0120003E4DF
:104FA300FF120003E490020EF0126DD4500E126D46
:104FB300E112000390020EE004F080ED7FC01200C6
:104FC300037FC0126E4DE4FF126E4DE490020EF0AB
:104FD300126DD4500E126DE1126E4D90020EE0046C
:104FE300F080ED7FC0126E4D12387AD2A012694E56
:034FF3000255CE96
:0E4FF6007BFFE4FD123AF97B017A00798022FC
:103D4F00EF2430F07C037DE8AF03AE0212037B7CDF
:103D5F00007D0A12037BED2430A3F07C007D64AF5D
:103D6F0003AE0212037B7C007D0A12037BED24302D
:103D7F00A3F07C007D0AAF03AE0212037B7C007DB3
:103D8F000A12037BED2430A3F022FFE4F0A3EFF03F
:103D9F0090021CE0FEA3E0FF7C007D5B120369AA8A
:103DAF0006AB0790021AE0FEA3E0FF7C207D5912BC
:103DBF000369EF2BFFEE3AFE90021FE02FFF9002F8
:103DCF001EE03ECF249BFBEF34A1FA7F0122744308
:103DDF009002DAF090027EE022900210E0248AF541
:103DEF0082E43402F583229002DA7453F090027E5B
:103DFF00E02275F00A84E5F0243022EFF0900210F3
:103E0F00E004F02274002FF582E43400F583E02201
:103E1F00F583E090021CFFE4F0A3EFF022F583E0BE
:103E2F0024E4900211F02224E4FFE034FFFE7C0032
:103E3F007D0A22F583E090021AFDE4F0A3EDF02253
:103E4F00F583EEF090020FE004F0227D0A7C00AFC4
:103E5F0003AE02222405F582E43400F583E02275D7
:063E6F00F00A8424302259
:106D6800125CD712654AEF70091263B3E49002B758
:0C6D7800F022120E489002B77401F022C5
:10654A007F06E4FE123E1320E00E74072FFF0EEEC4
:10655A00D3940840EF7F00220F0F0F123E13FEB4B0
:10656A0027047D0180027D00EEB460047E01800272
:0E657A007E00EE4D60069002CFEFF0227F0013
:0165880022F0
:100E4800E490027EF09002BAF09002897457F09014
:100E58000000E0C313FFE4FD122E4690027FEFF07E
:100E68009000017D011211F3900280EFF0900002D2
:100E78007D021211F3900281EFF09000037D0312BE
:100E880011FB900282EFF0A3742EF09000047D0411
:100E98001211FB900284EFF0900005E0C313FF7D70
:100EA80005122E46900285EFF0E4A3F0900294E03C
:100EB8009002B9F0900289E09002B8F09002CFE079
:100EC800FD2401F582E43400123E2C9002BAE0B40D
:100ED8006407900211E02464F0900211E0FFC394CB
:100EE800B4400AEFD394BD5004E024B0F09002114E
:100EF800E0FFC394BE400AEFD394C75004E02442F5
:100F0800F0900211E0FE75F064842430900274F0D1
:100F1800EE75F00A84123E01A3F0900211E0123E31
:100F280001900276F074022DF582E43400123E2C12
:100F3800C3943C4004E024C4F0900211E0FD123E4A
:100F48006E900277F0ED123E01A3F0A3742EF0909C
:100F580002CFE0FD2403F582E43400123E2CE0FECB
:100F6800123E6E90027AF0EE123E01A3F0E4A3F076
:100F780074042DF582E43400F583E0900214123EE7
:100F8800259002CFE0123E63FF7E00900216EEF03D
:100F9800A3EFF024E4FFEE123E3A12037BAA06AB5D
:100FA80007900215E0900214123E36120369EF2BE7
:100FB800FFEE3AAB07FAC3EB9420EA9403400874B7
:100FC800E02BFB74FC3AFAAD03AC02E41201517B4E
:100FD800F67A287994784112004612018AAA06AB5B
:100FE800077C277D1012037B9002D0123D4FA3741B
:100FF8002EF0123E5A123D90E4A3F0900210F090A9
:1010080002D0E06430702C90020FF090020FE0FFE5
:1010180024D1F582E43402F583E0FE74D02FF58202
:10102800E43402123E4FE0B407E1123E0CE0D394E0
:101038000240CC9002CFE0FF123E63900216123EAF
:101048004874062FF582E43400F583E0FF90021817
:10105800E4F0A3EFF0900217E0900216123E361269
:10106800037B7E007F64120369900219E024E4FD8B
:10107800900218E034FFCD2FFBED3EFAC3EB9490BD
:10108800EA9401400874702BFB74FE3AFA7D6412EE
:101098003E5C12037BEF24309002BB123D80123E6F
:1010A8005A123D90E4A3F0FF9002CFE0FE240CF525
:1010B80082E43400F583E0F9647D702A74092EF522
:1010C80082E43400123E42740A2EF582E43400129F
:1010D8003E1F9002CFE0240BF582E43400F583E054
:1010E80090021E123D999002CFE0FE240DF582E495
:1010F8003400F583E0647D701B740A2EF582E434B5
:1011080000123E42740B2EF582E43400123E1FE9B1
:10111800A3123D99EF640170537C277D10AF03AE95
:101128000212037B9002C5123D4FAE02AF03123D7F
:101138008CE4A3F0900210F09002C5E06430702CAB
:1011480090020FF090020FE0FF24C6F582E434020B
:10115800F583E0FE74C52FF582E43402123E4FE0B9
:10116800B406E1123E0CE0D3940340CC9002CFE0E9
:101178002407F582E43400F583E0900295F0E490CA
:101188000210F090020F7407F090020FE0FFC39472
:101198000D501A123E13C313900211F06420600818
:1011A800E0FF123DE8123E0A123E5380DC90000D2B
:1011B800E0541EC313FFD394004029123DE8742D58
:1011C800123E0BEFC3940AEF50044430800F123ED6
:1011D8006EFE123DE8EE123E0BEF123E01FF123D8D
:0A11E800EB123E0A123DE8E4F0FFAE
:1011F20022E0C313FF122E4622E0C313FF122E4633
:0112020022C9
:102E4600EFC39430402CEFD394395026AE07ED7083
:102E56000122EDB40103AF0622EDB40203AF062250
:102E6600EDB40302802BEDB404028031EDB405020B
:102E76008036EF644C70397E20ED70037F2022EDA2
:102E8600B40103AF0622EDB40203AF0622EDB4038C
:102E9600089002947453022FDDEDB40407E4900207
:102EA600BA022FDDEDB405089002897445022FDDC4
:102EB600EFC394414041EFD3944A503BEF24EFFED9
:102EC600ED7008123DDD2404022FDDEDB401081279
:102ED6003DDD2402022FDDEDB40207123DDD0402C2
:102EE6002FDDEDB40303AF0622EDB40403AF0622D3
:102EF600EDB40503AF0622EF644B70397E20ED700A
:102F0600089002DA7443022F9EEDB40108123DDDEB
:102F16002402022FDDEDB40207123DDD04022FDD8F
:102F2600EDB40303AF0622EDB40403AF0622EDB4FD
:102F36000503AF0622EFC39450404EEFD394595089
:102F460048EF24E0FEED700A7453123DDF240402BC
:102F56002FDDEDB40108123DF62402022FDDEDB49B
:102F66000206123DF604806FEDB4030790029474D6
:102F76004E8064EDB404079002BA74648059EDB4CF
:102F860005079002897457804EEF645A704D7E2073
:102F9600ED70109002DA7453F090027EE02404F093
:102FA6007F2022EDB40107123DF624028029EDB4FC
:102FB6000206123DF604801FEDB4030790029474D6
:102FC6004E8014EDB404079002BA74648009EDB41F
:0D2FD60005099002897457F0AF06227F4F65
:012FE30022CB
:105F8700F8900244E0FCA3E0FDA3E0FEA3E0FF12CB
:105F97000487E47B0AFAF9F8120487EB2430FF90B0
:105FA700024CE0244AF582E43403F583EFF09002D3
:105FB7004CE004F0E0244AF582E43403F583227BC5
:105FC700E87A03F9F8900244E0FCA3E0FDA3E0FEC1
:0E5FD700A3E0FF020487F090024CE004F022E9
:0D6FBA00759180759280759D8075BCA02238
:10672D00E4F5BDF5BEE5BC54E044084FF5BC0000F2
:10673D0000007DFAE5BC30E41753BCEFAFBDEF753B
:10674D00F004A4FFACBEEC7A002FFFEA35F0FE2278
:06675D00DDE27E037FFF78
:016763002213
:1051E0007F0712672DE4FCFD900248120538E47F2A
:1051F000E87E80FDFC900248E0F8A3E0F9A3E0FA25
:10520000A3E0FB1203FCE4FB7A24F9F8120487EF15
:105210002423FFE43EFEE43DFDE43CFC9002441206
:105220000538E4125FC6E4FBFAF9F8C312052770EB
:105230000890024CF07B64801BE490024CF0125FFB
:10524000C6EF2430FF90024C125FBBEF125FDDE42B
:105250007B64FAF9125F87742E125FDDE47B0AFA31
:10526000F9125F877456125FDD90024C125FBBE447
:03527000125FDDED
:015273002218
:10679800C313F04480F0A3E004F0E022E4F5D875D8
:1067A800F9FD75E908D2DE227B017A0079009001B3
:1067B80000E022900362E0640322F583E0FF900387
:0467C8007AE06F22E2
:1069A800308303D2C022C2C07F827E01126E6490FF
:1069B8000363EFF0C2AC12527490020DEFF0126E46
:0B69C800A890020DE0B40103124F5331
:0169D30022A1
:105274001259CF1267BB60037F0022900364E0647D
:105284007E60037F0022125A44900364E0FEB47EE1
:10529400081267BB60F07F0022E4900100F0E02474
:1052A40000F582E43400F583EEF0900100E004F0B0
:1052B400125A441267BB60037F0022900100E0FE93
:1052C400D3947840037F0022900364E0FF74002E9F
:1052D400F582E43400F583EFF0900100E004F0EF90
:1052E400B47ECD900366E070C7900100E014F01224
:1052F4006644BF01037F0122126895BF01037F0149
:04530400227F0022E2
:106644001267B024FEFD125C03900100E0FE24FEFC
:10665400F582E434FF1267C260037F002274FF2EC8
:10666400F582E434FFF583E0FF900379E06F600383
:0D6674007F0022900100E024FEF07F012253
:106895001267B014FD125C03900100E024FFF5823D
:1068A500E434FF1267C260037F0022900379E0643D
:0F68B5007E60037F0022900100E014F07F01223B
:1059CF00E4900362F0900364F0A284920DA3F09030
:1059DF00020EF0126F2D900364E0FFC313F0A3E0EB
:1059EF00B4061690020EE004F0E0B4030C900362CC
:1059FF007403F0E4900365F022E4900365F0C20EA7
:105A0F00200ED012704620DF183083079003627487
:105A1F0004F022A284300D01B350EBA284920DD278
:105A2F000E200EDC900364E0126798B407D2900347
:045A3F00627405F098
:015A43002240
:105A4400E4900366F090020EF090020EE0C3940816
:105A5400506212704620DF1E308307900362740484
:105A6400F022A284300D01B35008A284920DD20E0C
:105A74008004C20E80DF200E14900364E0FF1267DE
:105A840098B407079003627405F022801F126F2DEB
:105A9400900365E0B4050BA37401F0E4900365F092
:105AA40080A7900364E0C313F0E4A3F090020EE037
:045AB40004F08095E5
:015AB80022CB
:0E43A70090021FEBF0A3EAF0A3E9F0A3EDF003
:1043B500C2AC7F807E01126E64900225EFF0C2864A
:1043C500D287D282D285E4900365F0900223F090E3
:1043D5000225E02401FFE433FE900223E0C39FEEB3
:1043E5006480F87480985014E4A3F0124491E0C3FB
:1043F500942640F7900223E004F080D3E490022451
:10440500F0900222E0FF900224E0C39F5024900226
:104415001FE0FBA3E0FAA3E0F9120301FF12619C80
:10442500900220E475F0011203D0900224E004F01C
:1044350080CF90037AE0FF12619C900379E0FF1230
:10444500619CE4900224F0124491E0C3940540F786
:10445500D286C287C282126EA87F817E01126E64E7
:10446500900226EFF0D394004021E4900224F090CE
:104475000226E0FF900224E0C39F500F7F057E00D7
:0B448500126D12900224E004F080E4AD
:0D449000227F7E12619C900224E004F02245
:05619C00900227EFF066
:1061A100BF7E04D20C8002C20CE4900228F090025F
:1061B10027E05401FF7004B2858013900365E00469
:1061C100F0E0B4050D200C0A127032B285E49003A0
:1061D10065F0900227E0FFC313F01270329002289D
:0961E100E004F0E0C3940840C59D
:0161EA002292
:077032001267A430DFFD220C
:047046001267A42207
:0F6F2D00E4F5D875F9FE75E980D2DE30DFFD227C
:07703900C282D286C2872249
:10694E007F8F7E01126E64EF60227F1C7E02EF1F2E
:10695E00AC0670011E4C6012B2C3E4F5D875F9FF97
:0C696E0075E956D2DE20DFE680FBD2C3C4
:01697A0022FA
:1024C800000011892312329B462457AD653674BF2C
:1024D8008C489DC1AF5ABED3CA6CDBE5E97EF8F7DC
:1024E800108101083393221A56A5472C75B7643E0C
:1024F8009CC98D40BFDBAE52DAEDCB64F9FFE876BC
:102508002102308B02101399672676AF443455BDEB
:10251800AD4ABCC38E589FD1EB6EFAE7C87CD9F59B
:102528003183200A1291031877A7662E54B5453CCB
:10253800BDCBAC429ED98F50FBEFEA66D8FDC9747B
:102548004204538D6116709F042015A9273236BBAB
:10255800CE4CDFC5ED5EFCD7886899E1AB7ABAF35B
:102568005285430C7197601E14A1052837B3263A8B
:10257800DECDCF44FDDFEC5698E98960BBFBAA723B
:102588006306728F4014519D252234AB063017B96B
:10259800EF4EFEC7CC5CDDD5A96AB8E38A789BF11B
:1025A8007387620E5095411C35A3242A16B107384B
:1025B800FFCFEE46DCDDCD54B9EBA8629AF98B70FB
:1025C80084089581A71AB693C22CD3A5E13EF0B72B
:1025D800084019C92B523ADB4E645FED6D767CFFDB
:1025E80094898500B79BA612D2ADC324F1BFE0360B
:1025F80018C109483BD32A5A5EE54F6C7DF76C7EBB
:10260800A50AB48386189791E32EF2A7C03CD1B5EA
:10261800294238CB0A501BD96F667EEF4C745DFD9A
:10262800B58BA40296998710F3AFE226D0BDC134CA
:1026380039C3284A1AD10B587FE76E6E5CF54D7C7A
:10264800C60CD785E51EF497802891A1A33AB2B3AA
:102658004A445BCD695678DF0C601DE92F723EFB5A
:10266800D68DC704F59FE41690A98120B3BBA2328A
:102678005AC54B4C79D7685E1CE10D683FF32E7A3A
:10268800E70EF687C41CD595A12AB0A3823893B16A
:102698006B467ACF485459DD2D623CEB0E701FF91A
:1026A800F78FE606D49DC514B1ABA02292B983304A
:1026B8007BC76A4E58D5495C3DE32C6A1EF10F78FA
:055C030090021FEDF00E
:105C080074FFA3F0A3F090021FE0D39400403F126A
:105C18000301FF900220A3E06F25E0FFE433FE7448
:105C2800C82FF58274243EF583E493FC740193FD38
:105C3800900220E0FFECFEED6FFFEEF0A3EFF09096
:105C4800021FE014F0740129F9E43AFA80B89002CE
:105C580020E0FEA3E0F4FFEEF4FCEF90037AF0AE50
:065C680004EE900379F048
:015C6E002213
:106D1200EF4E6019EF1FAC0670011E4C600FE4F5D8
:0E6D2200D875F94CF5E9D2DE20DFE980FB22BE
:0E6F68000D0A444947492D3E5246203A20006A
:105F2800EE2402FFE433FE7C007D07120369AC0611
:105F3800AD0722900216E02417F582E43402F583B7
:105F48002274062DF58274003CF583222400F58224
:105F5800E43400F583227B017A007900900100E0A7
:105F6800FD2290020FE0FFA3E0FEC39F22F0900203
:0F5F780013E004F0222418F582E43402F58322AA
:1055CE007F0DE490020FF074002F125F56E020E082
:1055DE001174072FFF90020FE004F0E0D394064001
:1055EE00E62290020FE0605DE4900211F09002104E
:1055FE00F0125F6A501B125F287FB07E01124A20A4
:10560E00BF02069002117401F0900210E004F080C7
:10561E00E0E4900210F0125F6A501B125F287FB711
:10562E007E01124A20BF02069002117401F0900210
:10563E0010E004F080E0900211E0B401087F0E1239
:05564E004688125E0415
:015653002234
:0E4A2000900212EEF0A3EFF0A3ECF0A3EDF085
:104A2E00E4A3F0900216E0FFC39406502C900213FC
:104A3E00E02FFF900212E03400FE126E64EF700859
:104A4E00125F3B7440F08009EF25E0FF125F3BEFF1
:104A5E00F0900216E004F080CAE4900216F0900284
:104A6E0016E0FFFD900215E02DFD900214E03400DB
:104A7E00FC74002DF58274003CF583E0FE74172F54
:104A8E00125F41E06E60037F0022900216E004F098
:104A9E00E0B406CA900214E0FCA3E0FD2406125F07
:104AAE004CE0FE541EC313FF70037F01221FEF253F
:104ABE00E0FF125F49EE54E1F0125F49E04FF0EF74
:104ACE007014900214E0FEA3E02406F58274003EFA
:084ADE00F583E04480F07F0243
:014AE60022AD
:05468800900212EFF0AA
:10468D00900100E0D394784003024776E49002163F
:10469D00F0A3F0FFFE126E64EF7003024776E49014
:1046AD000216F0A3F0900213F0900216E0FEA3E0C4
:1046BD00FF126E64EF25E0900215F070037440F068
:1046CD00900215E0FF900213E0125F7DEFF0900273
:1046DD0017E004F07006900216E004F0125F76E029
:1046ED00C3940640C47F877E00126E64EF25E044BC
:1046FD00E090021EF0900214E004F0900100E0FF43
:10470D00900215F0900212E014FEC3EF9E90021479
:10471D00F0E4900213F0900214E0FF900213E0C356
:10472D009F5020900215E0FF125F54E0FE74072F9A
:10473D00F582E43400F583EEF0900215E014125F7B
:10474D007580D3E4900213F0900213E0FF125F7DA9
:10475D00E0FE900212E02F125F54EE125F75E0B48E
:09476D0007E6900100E02407F0CA
:014776002220
:105E04007F887E01126E64900213EFF0D3940040F9
:105E140021E4900212F0900213E0FF900212E0C31A
:105E24009F500F7F057E00126D12900212E004F065
:105E340080E4C2A1125F5E125C03125F5E1243A78C
:105E44007B017A007980122AB87BFF7A6F7968E443
:105E5400FD123AF97B017A007980E4FD123AF9D215
:015E6400A19C
:015E6500221A
:0F6F3C00E4F5D875F9FF75E940D2DE30DFFD22AC
:0F6F4B00E4F5D875F9FF75E9A0D2DE30DFFD223D
:106E3600C2C4126F3C7E08EFC313FF92C4126F3CAC
:076E4600DEF5D2C4026F3C2F
:106E4D00C2C4126F4B7E08EFC313FF92C4126F4B77
:076E5D00DEF5D2C4026F4B09
:1067CC0090021AEBF0A3EAF0A3E9F090021AE0FBB6
:1067DC00A3E0FAA3E0F9120301601790021AA3E4F4
:1067EC0075F0011203E6A9F0FA120301FF126E4DC7
:0367FC0080D9221F
:0970200090020DE0FF14F0EF22D4
:1060F30090020DEDF025E0F0EF24FE60160470260B
:10610300127020600BB2B77F017E00126D1280F017
:10611300D2B722127020600BB2967F017E00126DFF
:106123001280F0D296221270206011B2B7B296B2EA
:10613300A0B2A17F017E00126D1280EAD296D2B77F
:05614300D2A1D2A02250
:106A560041542B4E414D4547572D313030300D0AAC
:106A6600002047572D313030302046573A20312EFE
:0B6A760030392000563A312E30390034
:1069D40090033AE508F0A3E509F02290033CE50AA8
:1069E400F0A3E50BF022900338E50CF0A3E50DF0DD
:0C69F40022900336E50EF0A3E50FF02220
:106E9200125D3CC2B6126A001270041269A8125B3B
:066EA20096126DEE80EF78
:106B780020A2237F017E00126D1220A2191220612B
:106B8800C2AFC2A0C2A130A2FD7F017E00126D1269
:076B980030A2F375C72022B3
:10449D001268C4EF7010C2AFC2A0C2A1122061D2C7
:1044AD00A1D2A075C7207F801245857F00FEC00672
:1044BD00C0077F817E00126E64EFFDD0E02DF509FF
:1044CD00D0E03400F5087F827E00126E64EF7F002D
:1044DD00FEC006C0077F83124585FDD0E02DF50B8C
:1044ED00D0E03400F50A7F0012457BC006C007748A
:1044FD00010FFE126E64EFFDD0E02DF50DD0E0340E
:10450D0000F50C7F0212457BC006C0077F031245E4
:10451D008CFDD0E02DF50FD0E03400F50E7F831229
:10452D00458C7004D2A78002C2A77F907E01126EC7
:10453D0064EF7F00FEC006C0077F917E01126E649E
:10454D00EFFDD0E02DF511D0E03400F5101269D457
:10455D00C2001269DFC2011269EAC2041269F5C212
:10456D000390033EE510F0A3E511F0C202227E0197
:10457D00126E64EF7F00FE227E00126E64EF227ECB
:06458D0001126E64EF2232
:105D3C0043B70243B80243B710126B78127039752F
:105D4C00BBFFC2C4126CF412704A127040D2B7D2AC
:105D5C0096126FBA12449D126F84126FC7126FA005
:105D6C001242B012345A12345A7D027F031260F37D
:105D7C0012694EC28C9001017414F0C28CC28D75E4
:105D8C008C4CE4F58AD28CD2A9D2AF7BFF7A6A799B
:045D9C00560267FF45
:03000B0002494760
:10494700C0E0C0F0C083C082C0D075D000C000C036
:1049570001C002C003C004C005C006C007C28CC2A4
:104967008D758C4C758A00D28C900101E014F0E0B3
:104977006003024A057414F0E5094508601A9003BC
:104987003BE024FFF090033AE034FFF0E07002A32D
:10499700E070051269D4D200E50B450A601A90034E
:1049A7003DE024FFF090033CE034FFF0E07002A309
:1049B700E070051269DFD201E50D450C601A90031E
:1049C70039E024FFF0900338E034FFF0E07002A3F1
:1049D700E070051269EAD204E50F450E601A9003EC
:1049E70037E024FFF0900336E034FFF0E07002A3D5
:1049F700E070051269F5D203126F1C126CD6D0074E
:104A0700D006D005D004D003D002D001D000D0D03A
:094A1700D082D083D0F0D0E0324F
:10542900C0A80178FFFFFF00C0A801010008DC0146
:105439000203CDE9232E810F292392E5A2B67465D3
:105449007374000000303030000000333131312EE8
:1054590038314E000031323133312E323245004776
:10546900572D3130303020424541434F4E20000006
:10547900000000000000000000000000003331318E
:10548900312E37304E000031323133312E30304534
:105499000047572D31303030205758200000000088
:0F54A900000000000000000000000000000000F4
:1065890090022DE0FEA3E0FFE4FD126848E004F06C
:106599002290022DE004F02290022DE0FEA3E0FFFC
:1065A9002275C65A75C6A522ECF5C3AF058FC4225C
:0F65B90090022D7401F0A32290022DE4F0A32292
:1068C4007F1C1268EC60037F00227F1D1268EC6459
:1068D4000860037F00227F1E7E00126E64EF64DC7A
:0F68E40060037F00227F01227E00126E64EF228C
:0E6F7600E4F5C7F5C5F5C675C3FF75C4FF2267
:046E6400AD07AC06C4
:106E680075C78275C5011265B11265AA00AFC21255
:026E78006F7633
:016E7A0022F5
:106EE400AD07AC061265B175C78275C5031265AAF4
:036EF400026F76B4
:10697B00AD07AC0675C78275C5021265B11203016E
:10698B00F5C21265AA000DBD00010C740129F9E4D2
:0D699B003AFA900234E014F070E0026F76DA
:106832007F811268487F821268487F831268487F8E
:06684200841268487F8506
:10684800AB07AA0675C78275C502EAF5C3AF038F01
:0C685800C4AF058FC21265AA00026F7663
:10206100E4FFFE126EE47BFF7A54794790023474E8
:1020710007F0E4FF12697B7D0A7F071268487BFF46
:102081007A54794E9002347407F07F0912697B7A91
:102091005479299002347412F07F1012697B7A54BA
:1020A100793B900234740CF07F2212697BE4FD7F4E
:1020B1002E1268487F2F1268487F301268487F319E
:1020C1001268487F321268487F331268487F3412A1
:1020D10068487F351268487F401268487F801268DF
:1020E100481268327D0A7F871268487D217F8812F5
:1020F10068487D2F7F891268487D237F8A1268484E
:102101001265C17490F0E4FCEC90545493FD600EA0
:102111001265A1126593700312659A0C80EA12652B
:1021210089700312659A1265C174A0F0E4FCEC9009
:10213100545E93FD600E1265A112659370031265E2
:102141009A0C80EA126589700312659A1265C1744E
:10215100B0F0E4FCEC90546893FD600E1265A1129E
:102161006593700312659A0C80EA126589700312F7
:10217100659AE4FDFF7E01126848E404FF12684895
:102181007F021268487F031268487F041268487F03
:10219100051268487F061268487D0D7F071268485E
:1021A100E4FD7F0B1268487D3D7F081268487D2F52
:1021B1007F091268487D5F7F0A1268481265B97409
:1021C10010F0E4FCEC90548693FD600E1265A112B0
:1021D1006593700312659A0C80EA12658970031287
:1021E100659A1265B97420F0E4FCEC90549093FD6B
:1021F100600E1265A1126593700312659A0C80EA54
:10220100126589700312659A1265B97430F0E4FCA5
:10221100EC90549A93FD600E1265A11265937003C0
:1022210012659A0C80EA126589700312659A7D0124
:102231007F807E011268481D1268327F86126848CD
:102241007F871268480D7F881268481D7F89126850
:10225100487F8A1268487F8B1268487F8C126848D1
:102261007F8D1268487F8E1268480D7F8F126848F3
:10227100E4FCEC2490FFE43401FEE4FD1268480C18
:10228100ECB430EEE4FCEC24F0FFE43401FE7D30EC
:082291001268480CECB408EEE1
:012299002222
:0E6F92000D0A42542D3E52462F49533A20001C
:106EF7007B017A007900900100E0FD227B017A0096
:036F07007980226C
:0E6F8400759850758921758DFDD28E026EA80C
:106EA800C2ACC20FE4900206F07F80900186E4F045
:056EB800A3DFFCD2ACD9
:016EBD0022B2
:03002300025B2954
:105B2900C0E0C083C082C0D0309906C299C210803B
:105B390053309850C298300F07900206E4F0804421
:105B4900900206E02486F582E43401F583E599F0B4
:105B5900900206E004F0E599B4C01CE0D3940E402D
:105B690016900186E0B4C008A3E07004D20F801437
:105B7900C20F900206E4F0900206E0D3947E40043E
:0D5B8900C20FE4F0D0D0D082D083D0E03243
:105B9600300F69C2A1E4900100F07F02900206E096
:105BA60014FEEFC39E502174862FF582E43401F56E
:105BB60083E0FE74FE2FF582E434FFF583EEF09069
:105BC6000100E004F00F80D4126EF7125C03126E2F
:105BD600F71243A7126F03122AB8126F031240AAD4
:105BE6007BFF7A6F7992E4FD123AF9126F03E4FDB6
:0C5BF600123AF9D2A1E4900206F0C20FAE
:015C0200227F
:080003002010FDD2108F99229C
:1067FF0090021AEBF0A3EAF0A3E9F090021AE0FB83
:10680F00A3E0FAA3E0F9120301601790021AA3E4C0
:10681F0075F0011203E6A9F0FA120301FF1200034B
:03682F0080D922EB
:10585B000D0A4750532D3E4750524D43203A2020BE
:10586B00494F312020475053204E4F20636F6E6EAF
:10587B00656374210D0A000D0A4750532D3E4750A6
:10588B00524D43203A20000D0A4750532D3E4750AE
:10589B00524D43203A2020475053204E4F204C4F1F
:1058AB00434B210D0A004750532D3E4750524D4359
:1058BB00203A20004750532D3E4750474741203A4E
:1058CB002000244750524D43002447504747410086
:1028C700E0FAA3E0FB7C037DE8FFAE0212037BEF97
:1028D7002430FF90031FE024FDF582E43402F583E2
:1028E700EFF090031FE004F07C007D64AF03AE02BD
:1028F70012037B7C007D0A12037BED2430FFE0246A
:10290700FDF582E43402F583EFF090031FE004F055
:10291700E024FDF582E43402F583220F900371E091
:10292700FBA3E0FAA3E0F98F8275830002031AEF95
:102937002BFBEE3AFA7D0A7C00E024D0FFE434FF5B
:10294700FE020369EFF090031FE004F022900352A8
:10295700E0FBA3E0FAA3E0F922EF2BFFEE3AFEA398
:10296700E090031524D0FDEC34FFCD2FFFED3EF0B2
:10297700A3EFF022AA06AB077C037DE8E024D0FF93
:10298700E434FFFE020369A3F07B017A0179032295
:10299700900344E09002DEF0900345E09002DFF000
:1029A700900346E09002E0F0900347E09002E1F0E8
:1029B70090034822900345E09002DEF0900346E042
:1029C7009002DFF0900347E09002E0F0900348E0C8
:1029D7009002E1F090034922E0FAA3E0FB7C007D3E
:1029E7000AFFAE0212037B7C007D0A12037BED24F3
:1029F70030FF22900344E09002DFF0900345E0901F
:102A070002E0F0900346E09002E1F090034722EBEA
:102A1700F0A3EAF0A3E9F022E024D075F00AA4FFBE
:102A270022900343E02444F582E43403F583EEF077
:102A3700900343E004F00F22900344E09002E0F09B
:102A4700900345E09002E1F090034622EF75F00A0B
:102A570084E5F024302274552DF582E43403F583A0
:102A6700EFF00C0D22900317E0FEA3E0FF22900386
:102A770019E0FEA3E0FF2224D075F064A42FFFE045
:102A870024D02F22E0FF75F00A842430FE90031F24
:102A970022900344E09002E1F090034522E0FCA37A
:102AA700E0FDC39FEC9E22ED9FFFEC9EF0A3EFF0AD
:012AB70022FC
:0562D300900380EFF0D4
:1062D800E4F5AF9001847403F07F8C7E01126E6444
:1062E800EF7005759CFA8003759CFD43A21090031E
:1062F80080E024FF9208C207E4900185F0FF740350
:106308002FF582E43401F583E4F00F0FEFC3948096
:0563180040EC75AF012F
:01631D00225D
:106A81007F927E01126E64900312EFF024FE600E7D
:106A910014600E24027013300210C20280090250E9
:0B6AA10004126C0DBF010312554422CB
:106C0D003087037F00227F017E00126D12308703D3
:106C1D007F00223087FD7F017E00126D123087F3D9
:036C2D007F0122C2
:105EC800E4FF1262D3E4900381F020071E7F017E75
:105ED80000126D12900381E004F0E0D3942840EAA8
:105EE800E4F5AF7BFF7A58795B802EE4F5AF7BFF52
:105EF8007A587982FD123AF9122990E4FD123AF99A
:105F0800122990126AFFBF01091229901245937F46
:105F180001227BFF7A587992E4FD123AF97F002238
:10554400E4FF1262D3E4900382F02007071255BCF3
:1055540040F880407BFF7A5879B1E4FD123AF912A1
:105564002990E4FD123AF9122990126AFFBF011042
:105574001229901245931229901241B8D205800243
:10558400C2057F011262D3E4900382F0200709125E
:1055940055BC40F8E4F5AF227BFF7A5879BFE4FDAF
:1055A400123AF9122990E4FD123AF912299012479D
:0755B4007730050312486285
:1055BB00227F017E00126D12900382E004F0E0D393
:0355CB00942822FF
:105004009002F9E014601614605524026003025003
:10501400A7E4F5AF9002F904F0E4FF803F20070312
:105024000250AC7BFF7A5879B1E4FD123AF91229A7
:1050340090E4FD123AF9122990126AFFBF0110128E
:1050440029901245931229901241B8D2058002C2C8
:1050540005E4F5AF9002F97402F07F010262D330E7
:1050640007467BFF7A5879BFE4FD123AF91229907A
:10507400E4FD123AF9122990124777300610900293
:10508400FCE004F0E0D394054019C2068015300515
:1050940012124C6FBF010A124862D206E49002FC5D
:0950A400F08000E49002F9F02212
:1061EB00900103E064246007E4900185F0FF222016
:1061FB00081D90020A74FFF0A37458F074CD122995
:10620B008E1266BCBF0105D207E4F5AF7F0022906A
:10621B00020A74FFF0A37458F074D412298E12661C
:0F622B00BCBF0108D207E4F5AF7F01227F00223C
:106BE900E4900310F0A3F09002E5F09002E3F09036
:106BF90002FBF09002FAF0C2059002FCF0C2069086
:046C090002F9F0227A
:06477700900340122A1617
:10477D00E4FFFE900340122926FD6009B42C010EC2
:10478D000FEEB409EE900340122926642D70600FD0
:10479D00900343F0900340122926FE642E6005120B
:1047AD002A2880F07F069002DD7430F0A3DFFC90A4
:1047BD0002DD742DF0900343E024FE6013146015A8
:1047CD001460171460192404701A9003440247F4FE
:1047DD00122A988012122A3F800D1229FA8008128F
:1047ED00299780031229BBE09002E2F002485CE4B5
:1047FD00900343F0900340122926FE642E600512AB
:10480D002A2880F07F069002DD7430F0A3DFFC9043
:10481D000343E024FE601314601614601814601A2C
:10482D002404701B900344024857122A98024857DB
:10483D00122A3F80151229FA8010122997800B90A9
:10484D000344E09002DDF01229BBE09002E2F0E4B7
:04485D009002E3F0F2
:014861002234
:066AFF0090036E122A163E
:106B0500E4FFFE90036E1229266009B42C010E0FD6
:106B1500EEB402EF90036E122926B441037F0122E1
:026B25007F00EF
:016B2700224B
:06459300900371122A16CC
:10459900E4FFFE1229236009B42C010E0FEEB403C7
:1045A900F2E4FE122923FD642E600C74FD2E1229FB
:1045B9001AEDF00E0F80EC90037112295774FD2E3D
:1045C90012291AEDF00E0F12292EFD74FD2E122953
:1045D9001AEDF00E0F12292EFD74FD2E12291AED77
:1045E900F00E0F122923642C60030F80F612292282
:1045F900FD74FD2E12291AEDF00E0F74FD2E1229ED
:104609001A742FF00E122923642C60030F80F60F01
:10461900122923FD642E600C74FD2E12291AEDF067
:104629000E0F80EC90037112295774FD2E12291A6E
:10463900EDF00E0F12292EFD74FD2E12291AEDF040
:104649000E0F12292EFD74FD2E12291AEDF00E0FF0
:10465900122923642C60030F80F6122922FD74FDB0
:104669002E12291AEDF00E74FD2E12291AE4F07F8C
:0E467900997E01126E64BF01031218D37F01F7
:014687002210
:1018D3009002FD122A1FA3E024D02F90031BF09047
:1018E30003007D6412293E9002FF12297B900302BC
:1018F300122936EF2BFFEE3AFEA3E09003131229D1
:101903006B900304E090031DF0E490031FF0900339
:101913001F122917E0642F600512294D80F0122948
:101923004DE4FF90031F122917E0642E600612296D
:101933004D0F80EFEF24FB603504707590030612A2
:101943002A1FA3E024D02F90031CF09003097C00EE
:101953007D64122983AA06AB0790030812297F909E
:10196300030B12293612296090030D0219AF90035D
:1019730007122A1F900306E0900308122A7E9003A1
:101983001CF090030AE024D0FFE434FFFE7C007DCA
:101993006412036990030912297BEF2BFBEE3AFAD9
:1019A30090030C12293C12296090030EE090031E51
:1019B300F07F9B7E01126E64900317E4F0A3EFF0B7
:1019C3007F9A7E01126E64BF0130122A6C90031459
:1019D300E02FF0900313E03EF0C3A3E09470900374
:1019E30013E09417404BA3E02490F0900313E034EA
:1019F300E8F090031BE004F08037122A6C90031385
:101A0300122AA44008900313122AAE8024900314D0
:101A1300E02470F0900313E03417F0122A6CC390A3
:101A23000314E09FF0900313E09EF090031BE01477
:101A3300F07F9D7E01126E64900319E4F0A3EFF032
:101A43007F9C7E01126E64BF0130122A75900316CB
:101A5300E02FF0900315E03EF0C3A3E094709003F1
:101A630015E09417404BA3E02490F0900315E03465
:101A7300E8F090031CE004F08037122A75900315F8
:101A8300122AA44008900315122AAE80249003164C
:101A9300E02470F0900315E03417F0122A75C39018
:101AA3000316E09FF0900315E09EF090031CE014F2
:101AB300F0E490031FF090031B122A8B122917EEF8
:101AC30012294C122A53FF12291712294B90031380
:101AD3001228C7742E12294C9003131229DF900386
:101AE3001F12291712294B7C007D0AAF03AE021285
:101AF30029F212291712294B90031DE0FF90031FAF
:101B0300122905742F12294C90031CE0FFD3946310
:101B1300401EE0FE75F064842430FD90031F1229FB
:101B230017ED12294CEE75F00A84122A54FE800632
:101B330090031C122A8B122917EE12294C122A53D6
:101B4300FF12291712294B9003151228C7742E125E
:101B5300294C9003151229DF90031F12291712290C
:101B63004B7C007D0AAF03AE021229F21229171231
:0F1B7300294B90031EE0FFA3122905E412294C11
:011B82002240
:104C6F009002E4E0F97002FF22900310E0FEA3E04F
:104C7F00FF9002DBE0FAA3E0FBD39FEA9E4008EB34
:104C8F009FFDEA9EFC80159002DBE0FEA3E0FFC3D0
:104C9F00900311E09FFD900310E09EFCD3ED94B4C0
:104CAF00EC9400401074689D90037CF074019C900C
:104CBF00037BF0800890037BECF0A3EDF0D390031F
:104CCF007CE0941990037BE094004006E49002FA94
:104CDF00803A9002FAE004F0E9C3940A500CE0C362
:104CEF0094324003E480257F00229002E4E0C394D5
:104CFF0032500F9002FAE0C3941E4003E4800D7F00
:104D0F0000229002FAE0C394144014E4F09002DB06
:104D1F00E0FFA3E0900310CFF0A3EFF07F01227F1D
:014D2F000083
:014D30002260
:0641B800900352122A16CA
:1041BE00E4FCFD1229548C821229306009B42C01C2
:1041CE000D0CEDB407ED1229548C82122930B42C4B
:1041DE0003E48041E4FD1229548C82122930FF64DD
:1041EE002E6005122A5D80EEED24FD601004701F16
:1041FE00900355122A1FA3E024D02F801890035647
:10420E00122A1F900355E0900357122A7E800690C3
:10421E000355E024D09002E4F01229548C82122926
:10422E0030642C60030C80F10C1229548C821229FC
:10423E0030B42C08E49002DBF0A3F022E4FD122946
:10424E00548C82122930FF642E6005122A5D80EE96
:10425E00ED24FD600C04703890035512293CA380A8
:10426E001B90035612293CAA06AB079003557D649A
:10427E00122940EF2BFFEE3AFE900357E024D0FDBB
:10428E00EC34FFCD2FFFED3E9002DBF0A3EFF022DA
:10429E00900355E024D0FEE434FF9002DBF0A3CE71
:0142AE00F01F
:0142AF0022EC
:1066BC00900207122A1690020A122957120301FFA0
:1066CC0060259002071229571203016F60037F00A7
:1066DC0022900208E475F0011203D090020BE475CD
:0A66EC00F0011203D080CF7F0122DD
:106C9600A3E02403F582E43401F583E59BF090013B
:106CA60085E004F022E02403F582E43401F583E470
:026CB600F022CA
:0300430002514A1D
:10514A00C0E0C0F0C083C082C0D075D000C000C02B
:10515A0001C002C003C004C005C006C007E59A30FA
:10516A00E106539AFD0251C5E59A30E04E539AFE84
:10517A00900184E064017015126C96E59BB40A0BE9
:10518A00126CAB126CA4126B51802B802490018498
:10519A00E064037021126C96900102E004F0E59B32
:1051AA00B40A0E900185126CAB126CA41261EB80EA
:1051BA0005126FEC8005900185E4F0D007D006D087
:1051CA0005D004D003D002D001D000D0D0D082D0F4
:0651DA0083D0F0D0E032AA
:0C6FEC00900185E0D3947E4002E4F02286
:0D6FC700E4F5A2759A50758E10759CF422A9
:100544004750532000B1B1CEB33A2000C4CFCEB34C
:100554003A2000B6ABBEAD3A2000CEF7BEAD3A208D
:1005640000BAA3B0CE3A20002020204757313030C3
:100574003020202000535441545553204F4B210028
:100584002020C6F8CFF3BDD3BFDAB0E52020002089
:10059400202020C3BBC1ACBDD3A3A120200057653C
:1005A40061746865722053746174696F6E004E6F74
:1005B40020636F6E6E656374696F6E2120005765EA
:1005C40061746865720025007061004449523A0004
:1005D4005753203A002F00204D2F5300524E203AFB
:1005E400006D6D00504F533A00202020004D5347BA
:1005F4003A005961636874004D6F746F00427573FB
:100604000041545600547275636B0056616E004885
:100614006F7273650042616C6C6F6F6E005472612F
:1006240063746F72004A65657000416E74656E6E26
:100634006100575800444947490043617200506CB7
:10064400616E650000001800240024F4190C0204F3
:1006540004000400040004000204010800F0000087
:10066400000000001028100000000000000000003E
:100674000000000020202020200020005050000016
:10068400000000005050F850F850500010385070DE
:1006940028287000006868102058580030283070EE
:1006A40048483000101000000000000010202020F6
:1006B4002020100020101010101020000020707056
:1006C40070200000002020702020000000000000A6
:1006D400001010000000007800000000000000007E
:1006E400000020000808101020204000304848482E
:1006F4004848300020602020202070003048081036
:10070400204078003048083008483000103030501D
:1007140050781000784040700808700030484070ED
:1007240048483000784808102020200030484830DD
:10073400484830003048483808483000000020005D
:10074400002000000000200000204000081020408D
:1007540020100800000078007800000040201008F5
:10076400102040003048081020002000304848582D
:10077400282838003048484878484800704848706D
:10078400484870003048404040483000704848486D
:10079400484870007840407040407800784040708D
:1007A4004040400030484058484830004848487865
:1007B40048484800702020202020700008080808BD
:1007C4004848300048485060504848004040404045
:1007D4004040780048787848484848004868685855
:1007E4005848480078484848484878007048487055
:1007F40040404000304848486858380070484870C5
:1008040060504800304840300848300078202020AC
:100814002020200048484848484830004848484874
:1008240030303000484848487878480048483030EC
:100834003048480088885020202020007808103054
:10084400204078003020202020203000808040404C
:100854002020100030101010101030002050000024
:1008640000000000000000000000780020200000CC
:100874000000000000000038384838004040407054
:100884004848700000000038404038000808083824
:1008940048483800000000307840300000102078CC
:1008A40020202000000000384838083040404070C4
:1008B40050505000000020002020200000001000B4
:1008C4001010106040404058605048002020202004
:1008D4002020700000000078585858000000007074
:1008E40048484800000000304848300000000070CC
:1008F4004848704000000038484838080000005854
:100904006040400000000038601870000000207053
:10091400202030000000004848483800000000480B
:1009240048303000000000A8A870500000000048C3
:100934003030480000000048483808300000007893
:10094400102078003020204020203000202020205B
:10095400202020006020201020206000285000006B
:100964000000000000707070707000004248345441
:1009740044562D31303E4150455435313A213331BE
:1009840033342E33314E2F31323032302E32324521
:10099400722031323320392E30560D0A00000059AE
:1009A40000003C00005500005600006B000076007B
:1009B400006500004F00004600006A00007200005D
:1009C4005F00002300003E000060FF05F6FF05FC09
:1009D400FF0601FF0605FF0609FF060FFF0613FFCA
:1009E4000619FF0621FF0629FF062EFF0636FF061D
:0709F40039FF063EFF064239
:1012030090022AE0FBA3E0FAA3E0F9900230E0F5B4
:101213008275830012031AFF90022EE02432F582B6
:10122300E43402F583EFF090022EE004F0900230F4
:10123300E004F090022FE004F0E02290022EE0247C
:1012430032F582E43402F583E4F0900233E024D0F3
:10125300FFE434FFFE7C007D0A120369AA06AB0794
:10126300900232E024D0FFE434FFFE7D6412036970
:10127300EF2BFFEE3AFE900234E024D0FDEC34FF76
:10128300CD2FFFED3EFEE4FD90023C120538E47FD6
:10129300FEFEFDFC90023CE0F8A3E0F9A3E0FAA314
:1012A300E0FB1203FCE47BE87A03F9F8120487906D
:1012B3000240120538900240A3A3E0FFA3E090028E
:1012C30038CFF0A3EFF0900238E0FAA3E0FB7C0004
:1012D3007D64FFAE0212037B7C007D0A12037BED6B
:1012E3002430900232F0AF037C007D0AAE02120379
:1012F3007B7C007D0A12037BED243022E02411F570
:1013030082E43402F583EEF090020DE004F0EF7511
:10131300F00A8475F00A84E5F02430FEE02411F528
:1013230082E43402F583EEF090020DE004F0EF75F1
:10133300F00A84E5F02430FEE02411F582E434025F
:10134300F583EEF090020DE004F02290022EE024EB
:1013530032F582E43402F583E4F0900233E024D0E2
:10136300FFE434FFFE7C007D0A120369AA06AB0783
:10137300900232E024D0FFE434FFFE7D641203695F
:10138300EF2BFFEE3AFE900234E024D0FDEC34FF65
:10139300CD2FFFED3EFE900238F0A3EFF022E024C4
:1013A30022F582E43403F583EFF0900321E004F0A7
:1013B300E02422F582E43403F58322900246E0FB25
:1013C300A3E0FAA3E0F902030190021AFFF09002EE
:1013D30014E475F0010203D090024CE0FEA3E02474
:1013E30070F58274063EF583E49322EFF0A3EDF0EB
:1013F300A3EBF0A3EAF0A3E9F022900230F0E4902B
:10140300022FF02224E0FFE434FFFEEF7803229062
:101413000210E02400F582E43400F583E022FD901D
:101423000221E02422F582E43402F5832290024A69
:10143300E004F0E004F0900249E004F02290021787
:10144300E004F0E004F0900216E004F022EFF090E4
:101453000321E0042290022EE02432F582E43402D8
:10146300F583E4F022F0900214E0900213F090026E
:1014730015E0900214F0A3742AF0900211E0229078
:101483000221E004F0E004F0900220E004F0227D69
:10149300A11203690C7D6812037BA3EEF0A3EFF0A6
:1014A30022FF90024AE0244EF582E43402F583EFF2
:1014B300F090024DE004F022FF900217E0241CF5A7
:1014C30082E43402F583EFF090021BE004F022A3E0
:1014D300F0900238E0FEA3E0FF2274FD2FF582E4D2
:1014E3003402F583E0FF90032122900233F07C0065
:1014F3007D0AAF03AE022290023A7D0AE0FAA3E02E
:10150300FB7C00FF227420F090023AE0FEA3E0FF90
:101513002290024CFFEEF0A3EFF022E490024AF097
:10152300900249F022E4900217F0900216F022E4B0
:10153300900321F090032022900211E0FFA3E0FD2D
:1015430090021AE0FB22E0900212F0E4A3F0900272
:1015530011E022EF25E0FF0EEE22F0900320E004DD
:10156300F022900234F0E4A3F0900232E0227D01F5
:101573007BFF7E007F2D0202DB900320E0FFC3226E
:10158300FD7B017A0279127F0222E4900221F0901E
:041593000220F02220
:102C80007F337E00126E64EF64016003022E2D7F9D
:102C90008D7E01126E64EF7003022E2D7F3012586C
:102CA000DB7F011258DB7F0A7E00126D9F7F0612C8
:102CB00058DB7F0C1258DB12631E7BFF7A057944C8
:102CC000E4FD7F01125DA0E4900321F09002DB7D22
:102CD000641214FFAE0212037BEF2430FF90032135
:102CE0001213B31214501212E8FF1213B31214503D
:102CF000F09002DBE0FEA3E0FF1212F4FF9003214C
:102D00001213A174201213ACE4F07D03122E2E9046
:102D100002E4E0FF7E007C007DB91203697D64124D
:102D2000037BAB07AA06E4900321F0FC7D6412123A
:102D3000F1FF1213B31214501212E8FF1213B31260
:102D40001450F0AE02AF031212F4FF1213A1744B31
:102D50001213AC746D1213ACE4F07D05122E2E7BB1
:102D60000E7D08E4FF125FE5900304E07BFFB44EA4
:102D7000067A05794980047A057950E4FD7F0212CC
:102D80005DA0121532F012157C9407500E1214DD5E
:102D90001213B312145012155D80EB90032112131D
:102DA000B3E4F07F02122E3A90030EE07BFFB445AD
:102DB000067A05795780047A05795EE4FD7F03126F
:102DC0005DA01215327409F012157C9411500E1288
:102DD00014DD1213B312145012155D80EB90032111
:102DE0001213B3E4F07F03122E3A7BFF7A05796564
:102DF000E4FD7F04125DA0121532F012157C9406DA
:102E0000501674DD2FF582E434021214E51213B368
:102E100012145012155D80E39003211213B3E4F0F5
:0D2E20007B017A0379227D037F04125DA0FF
:102E2D00227B017A0379227F01125DA0227B017A38
:092E3D000379227D03125DA0223D
:1042B0007F337E00126E64EF640160030243A61236
:1042C0006B287F011258DB7F0A7E00126D9F7BFFF7
:1042D0007A05796C7F011261487BFF7A6A797A7F6F
:1042E00002126148E490020EF090020EE0FFC394C7
:1042F00010501474112FF582E43402F583E4F09029
:10430000020EE004F080E290020FE4F0A37410F0DB
:10431000FF7E00126E64E490020DF0EF75F064848D
:104320002430FE1212FF900210E004F0700690029A
:104330000FE004F0E490020EF090020DE02411F57D
:1043400082E43402F583742E12134690020FE0FECD
:10435000A3E0FF126E64EF75F064842430FE9002D7
:104360000D1212FF900210E004F0700690020FE0B0
:1043700004F090020EE004F0E0C3940340BB7B0124
:104380007A0279117F041261481251E07B017A03AD
:10439000794A7D047F02125DA07BFF7A0579797DE1
:0643A000017F03125DA085
:0143A60022F4
:0915970090022A1213F4A3EDF0F6
:1015A0007F337E00126E64EF640160030218827F55
:1015B0000B7E01126E64EF70030218827F301258A6
:1015C000DB7F011258DB7F0A7E00126D9F7F0612BF
:1015D00058DB7F0C1258DB12631E90022DE0702B3B
:1015E0007BFF7A057984FD7F01125DA07BFF7A0580
:1015F00079937F021218CB7A0579A27F031218CB58
:101600007A0579B2E4FD7F04025DA07BFF7A05795B
:10161000C2E4FD7F01125DA0E490022EF0740D1271
:1016200013FD121203B403FA12134EC39420EE9466
:101630000050151214D4C374209FF0E49E90023819
:10164000F0E4900231F08014900239E024E0F09050
:101650000238E034FFF09002317401F01214D47CAF
:10166000007D0A1203697D1212149A900231E07013
:1016700006A3742DF080069002327420F012150B30
:10168000C3940AEE9400500C9002337420F07C0056
:101690007D0A800F90023AE0FAA3E0FBFF1212EB02
:1016A0001214ED1212F8A3F0E4A3F07F011218A9AE
:1016B0007A067948E4FD7F071260437B0E7D08E4DB
:1016C000FF125FE5E490022EF074191213FD12125E
:1016D00003B402FA1214587B017A0279327D067F34
:1016E00002125DA07BFF7A0579CA7D077F02125D39
:1016F000A0E490022EF0900230741C12140012121A
:1017000003B404FA121458900232E0B43003742087
:10171000F07F031218A97A0579CC7D077F03125D4B
:10172000A01251E07B017A03794AE4FD7F09121887
:10173000B704121400121203B403FA1214589002E0
:1017400032E0B4300B7420F0A3E0B430037420F026
:101750007A0579CF7D081218C37D081218837405A5
:10176000121400121203B403FA12134E12149290C0
:1017700002327420F0C3EF940AEE9400500CA312CE
:1017800015081212F4900234800D1214FA1212EF9E
:101790001214ED1212F8A3F0E4A3F07BFF7A05799E
:1017A000D47D107F08123E757D10121883740912C3
:1017B0001400121203B403FA12134E121492C394BB
:1017C0000AEE9400500E9002321215081212F49094
:1017D000023380101214FA1212EF9002321214F037
:1017E0001212F8A3F0E4A3F07D101218977D107F79
:1017F0000D123E757BFF7A0579DB7D107F0E121886
:10180000B77411121400121203B403FA12123E122A
:1018100014D21212F4121565B4300B7420F0A3E048
:10182000B430037420F07A0579E07D181218C37B78
:10183000017A0279327D187F0A123E75E490022EF9
:10184000F09002307415121400121203B403FA124D
:10185000123E1214D21212F4121565B4300B742019
:10186000F0A3E0B430037420F07D181218977D18AF
:101870007F0D123E757BFF7A0579E57D187F0F128B
:021880003E75B3
:10188200227B017A0279327F0A123E75E490022E9F
:10189200F0900230227BFF7A0579D97F0C123E75D7
:1018A2007B017A027932227B017A0279327D05123A
:1018B2005DA07BFF22123E75E490022EF090023072
:1018C200227BFF7F08123E7522E4FD125DA07BFFA2
:0118D20022F3
:10387A007F337E00126E64EF640160030239BD7FFC
:10388A008B7E01126E64EF70030239BD7F301258CD
:10389A00DB7F011258DB7F0A7E00126D9F7F0612C2
:1038AA0058DB7F0C1258DB12631E90020F7408F06B
:1038BA002408FD7BFF7A0579E8E4FF123E75900241
:1038CA000FE02410FD7BFF7A0579EDE4FF123E75C7
:1038DA00E4FB7D107F08125FE57BFF7A0579F17DB5
:1038EA00027F081235BE7B017A02798A7F01126152
:1038FA0048E4900210F0FF74002F121418B4F00775
:10390A00900210EFF080050FEFB480EB900210E008
:10391A0004F0121415FFB427047E0180027E00EF22
:10392A00B460047F0180027F00EF4E60281239BE26
:10393A00FF2409F582E43400F583E0B42205EF247C
:10394A000D8006900210E0240AFF126D8490021086
:10395A00E02407805A121412FFB43D047E0180024B
:10396A007E00EFB421047F0180027F00EF4E6011D8
:10397A001239BE2414FF126D84900210E0241380C1
:10398A002E121412FFB440047E0180027E00EFB4AE
:10399A002F047F0180027F00EF4E60171250AD9016
:1039AA000210E0241BFF126D84900210E0241AFF1B
:0339BA001254B8EC
:0939BD00221250AD900210E0222C
:1050AD009002117408F07F0C900212E4F0A3DFFC63
:1050BD00E4FF747F2FF582E43402F583E0FE74146F
:1050CD002FF582E43402F583EEF00FEFB40CE3908C
:1050DD0002127420121468240812513D7F0C9002A4
:1050ED0012E4F0A3DFFCE4FF74742FF582E43402C4
:1050FD00F583E0FE74132FF582E43402F583EEF0B0
:10510D000FEFB40CE3900213E09002121214682416
:10511D001012513D9002B91215492408121583122F
:10512D003E759002B81215492410121583023E7572
:0D513D00FD7B017A0279127F03123E75227C
:106D840074002FF9E43400FA7B01900100E0C39F02
:0B6D9400900216F07D027F0A024DE81D
:0554B800900211EFF06D
:1054BD0078147C027A0979A112157178417C027AEF
:1054CD000979CE121571900211121415900213F074
:1054DD00E4900212F0900212E0FFC3940E504BEFD5
:1054ED0075F003A42414F582E43402F583A3E0FAE5
:1054FD00A3E0FF900213E0FD7C00EFB50524ECB5B1
:10550D000220900212E075F003A42441F582E434E8
:10551D0002F583E0FBA3E0FAA3E0F97D057F01022C
:10552D005DA0900212E004F080AB900213E0FB7DD1
:06553D00057F01126287E8
:015543002245
:07614800900221EF1213F297
:10614F007F301258DB900221E024FE600E14600FA6
:10615F00146010240370117F80800A7F9080067F67
:10616F008880027F981258DBE4900225F09002227B
:10617F001213C1FF60161259559002231213D490B7
:0C618F000225E004F0E0D3941040E2226E
:01619B0022E1
:085E6600900374EFF0A3EDF0CE
:105E6E007F301258DB900374E024FE60121460172A
:105E7E0014601C24037022900375E0248080169019
:105E8E000375E02490800E900375E02488800690C0
:105E9E000375E02498FF1258DBE4900376F090032C
:105EAE0076E0FFC394085011EF90066893FF1259E5
:095EBE0055900376E004F080E544
:015EC70022B8
:1062870090026EEFF0A3EDF0A3EBF07F301258DB36
:1062970090026EE024FE601214601714601C240341
:1062A700702290026FE02480801690026FE02490A5
:1062B700800E90026FE02488800690026FE0249899
:0C62C700FF1258DB900270E0FF025955F6
:065DA00090026E1213EEEA
:105DA6007F301258DB90026EE024FE6012146017FA
:105DB60014601C2403702290026FE02480801690E9
:105DC600026FE02490800E90026FE0248880069097
:105DD600026FE02498FF1258DBE4900273F0900201
:105DE600701213C1FF60161259559002711213D426
:0D5DF600900273E004F0E0D3941040E2222C
:015E0300227C
:066043009002441213EE6E
:10604900E4A3F07F341258DB900245E02480FF126C
:1060590058DB900244E02480FF1258DB7F3012584D
:10606900DB9002461213C1FF1259559002471213D1
:10607900D49002461213C1FF1259559002471213C8
:10608900D4900245E004F0900249E004F0E0C394A2
:036099001040B004
:01609C0022E1
:0A5FE500900245EBF0900244EFF04B
:105FEF00C3ED9F900247F0E4900246F0900247E025
:105FFF00FF900246E0C39F50367F341258DB900269
:10600F0045E02480FF1258DB900244E02480FF1209
:10601F0058DB7F301258DB7FFF1259557FFF125923
:10602F0055900244E004F0900246E004F080BD7FFA
:04603F00360258DBF2
:063E75009002441213EE5E
:103E7B001213BE7003023F3F900245E090024BF0DD
:103E8B00E4900249F0900249E0FFC3941050107483
:103E9B004E2FF582E43402F583E412143880E612D7
:103EAB0013BE121407C333CE33CED8F91215141226
:103EBB00151E1213DB1214A4700690024CE004F0D2
:103ECB00121430E0B408EB9002471213D41213BE55
:103EDB00701312151F123F44A3121436E0C394083B
:103EEB0040F3023F3F1213BE121407C333CE33CE3F
:103EFB00D8F912151490024A7401F0E4900249F0BB
:103F0B001213DB1214A4700690024CE004F012148E
:103F1B0030E0B408EB12151E123F44A3121436E026
:103F2B00C3940840F39002471213D4900244E00468
:093F3B00F0023E7B7F360258DBE8
:103F44007F341258DB90024BE02480FF1258DB9040
:103F54000244E02480FF1258DB7F301258DB9002C9
:103F64004AE0244EF582E43402F583E0FF12595509
:103F740090024AE004F0E0244EF582E43402F58332
:0C3F8400E0FF12595590024AE004F022C0
:064DE8009002111213EE0F
:104DEE00A3E07003024E9D900216E0FFC3139002E3
:104DFE0018F0EF5401A3F0E4900217F0900218E0BF
:104E0E00FF900217E0C39F50569002131213C11267
:104E1E0013CCEFC39420500690021A743FF0900208
:104E2E00131213C190021B1213CFEFC3942050061E
:104E3E0090021B743FF012153BA3E090021FF0127C
:104E4E004BAC900211E004F0E0D3940F40087408CC
:104E5E00F0A3E02408F0900217E004F0024E0A904E
:104E6E000219E060259002131213C11213CCEFC386
:104E7E009420500690021A743FF0E490021BF01238
:0F4E8E00153BE490021FF0124BAC7F361258DB3D
:014E9D0022F2
:084BAC0090021CEFF0A3EDF0F4
:104BB400E4900220F0900220E0FFC39410500C74A3
:104BC400222F121428E412148A80EAEB121407C369
:104BD40033CE33CED8F9FF12158D74702F1213E42F
:104BE400121421EDF00FBF00010E121482E0B4087C
:104BF400E990021FE0FD602D121407C333CE33CEBB
:104C0400D8F9FF9002217401F0E4900220F074704E
:104C14002F1213E4121421EDF00FBF00010E121431
:104C240082E0B408E912158D7F341258DB90021D1E
:104C3400E02480FF1258DB90021CE02480FF12580D
:104C4400DB7F301258DB121422124C63121425122B
:0E4C54004C6390021D121488E0C3940840CAFD
:0D4C620022E0FF125955900221E004F022DB
:0E35BE009002131213F4900211EFF0A3EDF03F
:1035CC00900218EFF0A3EDF09002131213C17003E8
:1035DC000236CEE4900216F0900216E0FFC394106F
:1035EC005010741C2FF582E43402F583E412144855
:1035FC0080E69002131213C1121407C333CE33CEDC
:10360C00D8F990021A12151712152890021A1213D3
:10361C00DE1214BB700690021AE004F0121440E0A3
:10362C00B408E89002141213D49002131213C17050
:10363C00151215291236D3900219121446E0C394B0
:10364C000840F10236CE9002131213C1121407C3B4
:10365C0033CE33CED8F9FF90021AEEF0A3EFF090F0
:10366C0002177401F0E4900216F090021A1213DEA5
:10367C001214BB700690021AE004F0121440E0B46D
:10368C0008E81215281236D3900219121446E0C31A
:10369C00940840F1900211E004F09002141213D43B
:1036AC00900211E0D3940F400E7408F0900219E0D0
:1036BC00900212F00235D4900212E0900219F0023E
:0736CC0035D47F360258DB04
:1036D3007F341258DB900219E02480FF1258DB90EC
:1036E3000211E02480FF1258DB7F301258DB900276
:1036F30017E0241CF582E43402F583E0FF125955E8
:10370300900217E004F0E0241CF582E43402F58310
:0C371300E0FF125955900217E004F0226C
:106B28007F301258DB7F01126B467F06126B467F5F
:106B38000C1258DB7F0A7E00126D9F02631E1258EA
:096B4800DB7F0A7E00126D9F2222
:10631E00E4900245F0E4900244F07F341258DB9092
:10632E000245E02480FF1258DB900244E02480FFF7
:10633E001258DB7F301258DBE4FF125955E4FF127E
:10634E005955900244E004F0E0C3941040CC900202
:0A635E0045E004F0E0C3942040BBCA
:016368002212
:1058DB00D2C1E4FEC2C500D2C5000EEEB405F5C2BE
:1058EB00C1C2C1C2C500D2C500C2C1C2C500D2C5AA
:1058FB0000C2C1C2C500D2C500E4FEEF30E704D23E
:10590B00C18002C2C1C2C500D2C500121556B40473
:10591B00EAC2C1E4FEC2C500D2C5000EEEB404F566
:10592B00E4FEEF30E704D2C18002C2C1C2C500D28F
:10593B00C500121556B404EAC2C1E4FEC2C500D2BA
:0A594B00C5000EEEB404F502702949
:10595500D2C1E4FEC2C500D2C5000EEEB405F5C243
:10596500C1C2C1C2C500D2C500D2C1C2C500D2C51F
:1059750000C2C1C2C500D2C500E4FEEF30E704D2C3
:10598500C18002C2C1C2C500D2C500121556B404F9
:10599500EAC2C1E4FEC2C500D2C5000EEEB404F5EC
:1059A500E4FEEF30E704D2C18002C2C1C2C500D215
:1059B500C500121556B404EAC2C1E4FEC2C500D240
:0A59C500C5000EEEB404F5027029CF
:106D9F00EF1FAC0670011E4C6010E4F5D875F9FCBE
:0B6DAF0075E966D2DE20DFE880FB22E1
:08702900E4FF000FEFB402FACE
:01703100223C
:1031670024309002C6F07C037DE8AF03AE02120361
:103177007B7C007D0A12037BED2430A3F090021ABA
:10318700A3E07C007D64FFAE0212037B7C007D0A16
:1031970012037BED24309002C8F07D0A7C00AF0358
:1031A700AE0212037B7C007D0A12037BED243022E2
:1031B700EF2BFFEE3AFEED39FDEC38FC9002C9A883
:1031C70004A905AA06AB07E075F00AA4FFE4FCFD15
:1031D700EB2FFBEA35F0FAED39F9EC38F8A3E0FF0D
:1031E700E4FEEB2FFFEE3AFEED39FDEC38FC22F55D
:1031F70083EEF075F001E49002110203D090021003
:10320700E0FBA3E0FAA3E0F9020301900214120520
:1032170038900214E0FCA3E0FDA3E0FEA3E0FFE486
:1032270012014C7BBF7A0E799C783E120046120140
:103237008A900214120538900214A3A3E0FFA3E0BA
:1032470090021ACFF0A3EFF090021AE02290021832
:10325700E0FF24C6F582E43402F583E0FE74C52F4F
:10326700F582E43402F583EEF0900218E004F022D0
:103277009002C77BE87A03E0FFE4FCFDFEF9F80261
:1032870003FC9002C8E0FFE4FCFDFE7B64FAF9F85A
:103297000203FC900213E0FFC322900213E004F044
:1032A70022120301FF740129F9E43AFA22FAA3E092
:1032B700FB7C277D10FFAE0202037B74C52FF582CE
:1032C700E43402227B017A007980229002CAF0E47A
:1032D700A3F0900219F022A3F090021AE0FEA3E0F7
:0232E700FF22C4
:105CD7007F0A90028AE4F0A3DFFC7F039002AAE424
:105CE700F0A3DFFC7F0A9002A0E4F0A3DFFC7F0AA9
:105CF700900296E4F0A3DFFC7F0A90027FE4F0A312
:105D0700DFFC7F0A900274E4F0A3DFFC7F0A9002B5
:105D1700BBE4F0A3DFFC7F0A9002D0E4F0A3DFFC32
:105D27007F0A9002C5E4F0A3DFFC7F0A9002ADE48E
:045D3700F0A3DFFCFA
:015D3B002245
:1063B3001232CB1263691232CB126E7B90020FEF53
:1063C300F07002FF2290020FE0FD2480F582E43496
:1063D30000F583E024D1601124F2600D24FD6009EF
:1063E300241F70101232CB80081232CB90020FE0C0
:0663F300FD12371F7F01BF
:0163F9002281
:106E7B00E4FF120301B43A04EF04FF221232AC0F09
:066E8B00EFB47DEE7F0074
:016E910022DE
:10636900E4FE1232A8EF643E6011748A2EF582E4CD
:106379003402F583EFF00EEEB40AE7E4FE1232A818
:10638900EFB42C047D0180027D00EFB43A047C0156
:1063990080027C00EC4D701174A02EF582E4340269
:0963A900F583EFF00EEEB40AD406
:0163B20022C8
:0B371F00900210EBF0A3EAF0A3E9F029
:10372A00AF058FF01231FD123204FF1231FAEFB4F5
:10373A0040047E0180027E00EFB42F047F018002E4
:10374A007F00EF4E6020E4900213F012329A940741
:10375A005014123204FE74962FF582E434021231A8
:10376A00F61232A180E5E4900213F012329A94071D
:10377A005014123204FE747F2FF582E4340212319F
:10378A00F61232A180E51232049002B91231F9120E
:10379A0031FAE4900213F012329A94085014123259
:1037AA0004FE74742FF582E434021231F61232A147
:1037BA0080E51232049002B81231F9123204FF90F5
:1037CA0002951231F9EF645F7003023879900210A2
:1037DA00E0FBA3E0FAA3E0F990000312031A642FB6
:1037EA006003023879900213F012329A940350144B
:1037FA00123204FE74BB2FF582E434021231F6123F
:10380A0032A180E51231FAE4900213F012329A944E
:10381A00035014123204FE74D02FF582E4340212DB
:10382A0031F61232A180E5124E9E123204642F70D4
:10383A003E90000112031A64417034900002120390
:10384A001A643D702A75F0011231FE1231FA1231F2
:10385A00FAE4900213F012329A9406500F123204CC
:0F386A00FE1232C21231F61232A180EA1232E996
:01387900222C
:104E9E00E4900214F0900214E0FFC39403501674D1
:104EAE00D02FF582E43402F583E024D0F090021482
:104EBE00E004F080E09002D012328C9002D11231D8
:104ECE00C6E412014C7BF67A28799478411200469A
:104EDE0012018AAB07AA067C277D1012037BEF24F2
:104EEE00309002D0F07C037DE81231A5A3F07D64F2
:104EFE001231A3A31231A0A3F0A3742EF0AE02AF11
:104F0E00031231ACA3F0E4A3F0FF9002D0E06430C2
:104F1E007032900214F0900214E0FE24D1F582E477
:104F2E003402F583E0FD74D02EF582E43402F5836D
:104F3E00EDF0900214E004F0E0B407DA0FEFD39432
:044F4E000240C72234
:014F5200223C
:1032E9009002C5E0642D600302337F90021804F058
:1032F900900218E0FFC39406500D1232C2F583E024
:1033090024D012326F80E9123277C004C005C0069A
:10331900C0079002C67B107A2712327ED003D002F2
:10332900D001D000EF2B1231EBC004C005C006C09C
:1033390007123289D003D002D001D0001231B7125E
:1033490032121232B4EF1231671232DE1231AC127C
:1033590032D29002C6E064306003023459900218F8
:1033690004F0123254E0B407F9900219E004F0E0D5
:10337900D3940340DD22E4900218F0900218E0FF94
:10338900C39406500D1232C2F583E024D012326F75
:1033990080E99002C6E0FFE4FCFDFE7B107A27F984
:1033A900F81203FCC004C005C006C0079002C5E0BE
:1033B900FFE4FCFDFE7BA07A867901F81203FCD0BC
:1033C90003D002D001D000EF2B1231EBC004C005AD
:1033D900C006C007123277D003D002D001D000EF67
:1033E9002B1231EBC004C005C006C007123289D0C8
:1033F90003D002D001D0001231B7123212FEA3E07D
:10340900FFE4FCFD7BA07A867901F8126486EF243B
:10341900309002C5F090021AE01232B47C007D0AA5
:1034290012037BED1231671232DE1231AC1232D245
:103439009002C5E064307018900218F0123254E01E
:10344900B407F9900219E004F0E0D3940440E122B2
:013459002250
:10004600EC4D6011E8497017ED33EC3304600DE4B4
:10005600FCFFFEFD22E933E8330470F80201F612D4
:1000660001C158046009E4CC2481500628500902D5
:1000760002002840030201FDC0E0EB4A7044B9804B
:1000860006D0E0FB0201ECEF4E701CBD8008EBFFD2
:10009600EAFEE9FD80EBE98DF0A4FEE5F002012F12
:1000A600E9CDF9EAFEEBFFEF89F0A4FCE5F0CE8995
:1000B600F0A42EFFE435F0CD89F0A42DFEE435F052
:1000C6008067EF4E7005BD80D780C3EF8BF0A4AC80
:1000D600F0EE8BF0A42CFCE435F0F8EF8AF0A42CBB
:1000E600E5F038FCE433CB8DF0A42CFCE5F03BF8CE
:1000F600EE8AF0A42CFCE5F038F8E433CF89F0A4BE
:100106002CFCE5F038CF3400CE89F0A42FFFE5F0C3
:100116003EFEE433C98DF0A42EFEE5F039CD8AF01B
:10012600A42FFFE5F03EFEE43DFD33D0E0FB500793
:100136000BBB000F020200EC2CFCEF33FFEE33FE8C
:06014600ED33FD0201D8BB
:10014C0075F020800E75F010800575F0087D007E2E
:10015C00007F003392D530D503120519EC334010D3
:10016C00EF33FFEE33FEED33FDEC33FCD5F0ED2237
:0E017C00E5F0247EA2D513CC92E7CDCEFF2273
:10018A00EDD2E7CD33EC3392D524814006E4FFFE6D
:10019A00FDFC22FCE4CFCECDCC24E0501174FF80CC
:1001AA00EDC3CC13CCCD13CDCE13CECF13CF047069
:0701BA00F030D5DE0205194B
:1001C100E9D2E7C933E833F892D5EDD2E7CD33EC84
:0701D10033FC5002B2D522FD
:1001D800EC30E7100FBF000C0EBE00080DBD000488
:1001E8000BEB6014A2D5EB13FCED92E7FD2274FF34
:1001F800FCFDFEFF22E480F8A2D574FF13FC7D808D
:03020800E480EFA0
:03000000026FF894
:0C6FF800787FE4F6D8FD758122026E92CD
:10020B00E709F608DFFA8046E709F208DFFA803ED5
:10021B0088828C83E709F0A3DFFA8032E309F608C2
:10022B00DFFA8078E309F208DFFA807088828C832A
:10023B00E309F0A3DFFA806489828A83E0A3F608DE
:10024B00DFFA805889828A83E0A3F208DFFA804CB8
:10025B0080D280FA80C680D4806980F2803380108F
:10026B0080A680EA809A80A880DA80E280CA8033F8
:10027B0089828A83ECFAE493A3C8C582C8CCC58370
:10028B00CCF0A3C8C582C8CCC583CCDFE9DEE78040
:10029B000D89828A83E493A3F608DFF9ECFAA9F0BF
:1002AB00EDFB2289828A83ECFAE0A3C8C582C8CC15
:1002BB00C583CCF0A3C8C582C8CCC583CCDFEADE2E
:1002CB00E880DB89828A83E493A3F208DFF980CC90
:1002DB0088F0EF60010E4E60C388F0ED2402B40489
:1002EB000050B9F582EB2402B4040050AF23234530
:0602FB00822390025B73F8
:10030100BB010689828A83E0225002E722BBFE02FA
:09031100E32289828A83E493222D
:10031A00BB010CE58229F582E5833AF583E0225098
:10032A0006E92582F8E622BBFE06E92582F8E222E2
:0D033A00E58229F582E5833AF583E49322FC
:10034700F8BB010DE58229F582E5833AF583E8F0EC
:10035700225006E92582C8F622BBFE05E92582C898
:02036700F22280
:10036900EF8DF0A4A8F0CF8CF0A428CE8DF0A42EA8
:02037900FE2262
:10037B00BC000BBE0029EF8DF084FFADF022E4CC66
:10038B00F875F008EF2FFFEE33FEEC33FCEE9DEC2F
:10039B00984005FCEE9DFE0FD5F0E9E4CEFD22ED75
:1003AB00F8F5F0EE8420D21CFEADF075F008EF2FBF
:1003BB00FFED33FD4007985006D5F0F222C398FDB0
:0503CB000FD5F0EA224D
:1003D000C5F0F8A3E028F0C5F0F8E58215827002B8
:0603E0001583E038F02255
:1003E600A3F8E0C5F025F0F0E582158270021583CA
:0603F600E0C838F0E82227
:1003FC00E88FF0A4CC8BF0A42CFCE98EF0A42CFCA0
:10040C008AF0EDA42CFCEA8EF0A4CDA8F08BF0A41D
:10041C002DCC3825F0FDE98FF0A42CCD35F0FCEB7C
:10042C008EF0A4FEA9F0EB8FF0A4CFC5F02ECD3941
:0F043C00FEE43CFCEAA42DCE35F0FDE43CFC22AE
:10044B0075F008758200EF2FFFEE33FECD33CDCC68
:10045B0033CCC58233C5829BED9AEC99E5829840EB
:10046B000CF582EE9BFEED9AFDEC99FC0FD5F0D6C8
:10047B00E4CEFBE4CDFAE4CCF9A88222B800C1B9F2
:10048B000059BA002DEC8BF084CFCECDFCE5F0CB30
:10049B00F97818EF2FFFEE33FEED33FDEC33FCEB69
:1004AB0033FB10D703994004EB99FB0FD8E5E4F924
:1004BB00FA227818EF2FFFEE33FEED33FDEC33FC11
:1004CB00C933C910D7059BE99A4007EC9BFCE99A05
:1004DB00F90FD8E0E4C9FAE4CCFB2275F010EF2F4A
:1004EB00FFEE33FEED33FDCC33CCC833C810D7074A
:1004FB009BEC9AE899400AED9BFDEC9AFCE899F885
:0E050B000FD5F0DAE4CDFBE4CCFAE4C8F92217
:10648600C2D5E830E70FB2D5E4C39BFBE49AFAE441
:1064960099F9E498F8EC30E717B2D51264BC120407
:1064A60087E4C39BFBE49AFAE499F9E498F880033D
:1064B60012048730D50DE4C39FFFE49EFEE49DFDE4
:0464C600E49CFC2234
:0E051900C3E49FFFE49EFEE49DFDE49CFC22F3
:10052700EB9FF5F0EA9E42F0E99D42F0E89C45F02A
:0105370022A1
:0C053800ECF0A3EDF0A3EEF0A3EFF02236
:00000001FF
